:0E000000802EFF02270EFFFFFFFFFF0224AE3F
:0300230002023B9B
:20002E00EC077581337508FF7509FF9095B2E4F0125FE980EDC82581C822C92581C97A0021
:20004E0022D083D082CF2581F581CFC082C08322CF2581F581CF22FBE0CB22FCE0FBA3E06C
:20006E00CC22FAE0F9A3E0CA2229F9E5F03AFA227C00CB30E7011CCB2275F00030E70215FA
:20008E00F022FDE493A3FEE493A3FF4E7009E493FE740193FF800BE493A3B5050BE493B539
:2000AE00F0068F838E82E473A380D8FEEBA4FD8EF0ECA4FCEB8EF0A4C5F02C2DC5F0221131
:2000CE00D38EF0ED22C002C001AAF0F97E007D007F11C3E933F9EA33FADF08F5F0E9D0019C
:2000EE00D00222ED33FDEE33FEC3ED9BF5F0EE9C40E0ADF0FED380DBBB000122C333C5F096
:20010E0033C5F0DBF722BB000122C3C5F013C5F013DBF722240280022401C5F03400C5F065
:20012E0022C394028003C39401C5F09400C5F0223134F4C5F0F4C5F02245F0702204223144
:20014E00964024801A3196401E7014801A3196400E7014800A3196500E800431AA6008E4C7
:20016E00F5F02231AA60F8E4F5F0042231AA40F780ED31AA40F170E780ED31AA40E170E7A6
:20018E0080DD31AA50E180D7C39BC5F09C20E70720D207C345F02220D2F9D322C5F0C39CCD
:2001AE007003E5F09B229095B2E0A360EEE0FFA3E0A3CF2582F582EF3583F58380EB7E008A
:2001CE00CF2508F582EE3509F583EF227E00CF2508F9EE3509FAEF227E00C5082FC508C533
:2001EE00093EC50922E4F520D201D200D203D205C2B4E4F50EF50DF50CF50BE4F512F5111F
:20020E00F510F50F74FFF513E588543FF588E589540FF5894420F5897450F598E58744801D
:20022E00F58774FAF58BF58DD28ED2AC22C0E0C0D0C083C082309839E50DB4FA028030506C
:20024E002E050DE50DB50E0280044002F50E908000C0E0E50B2582F582E43583F583D0E04E
:20026E00E599F0050BE50BB4FA004003750B00C298309948E511700DD200300235E4D5E0E1
:20028E00FDC2B4802DC20030011A300202D2B49080FAC0E0E5102582F582E43583F583D0C8
:2002AE00E0E0F59915110510E510B4FA004003751000C299200105200002D299D082D08389
:2002CE00D0D0D0E0322278FB120043E6C0E0B40A0B300308D204740D1581C0E0E511B4FAE9
:2002EE000280F950F7C2AC9080FAC0E0E50F2582F582E43583F583D0E0D0E0C0E0F00511EA
:20030E00050FE511B512004002F512E50FB4FA004003750F00300002D299D2ACD0E030044D
:20032E0008C204740AC0E080B322E4F5F078FB120043F608A6F022E51364FF7038E50D60D2
:20034E0034300531C2AC908000C0E0E50C2582F582E43583F583D0E0E0D2ACB40A030203E0
:20036E007374018010150D050CE50CB4FA004003750C0080C875F00022E4A20192E0F51F85
:20038E0070030203A8E5116003020393E4A20092E0F51FE51F700302039A22C2AC7513FF05
:2003AE007400F50CF50BC50DD2AC75F0002274FFC513B4FF2EE50D0060FBC2AC908000C02C
:2003CE00E0E50C2582F582E43583F583D0E0E0C0E0150D050CE50CB4FA004003750C00D274
:2003EE00ACD0E030050BB40A030203C3B40D02740A75F000221203BCC0E0C0E0C0E012023D
:20040E00D4D0E0D0E0D0E075F00022E51375F0007BFF7C00120169700302043174FFF5F092
:20042E0002044178FB120043E60886F0F51318E60886F02278FB1200438682088683E06074
:20044E0016C083C082C0E0C0E01202D4D0E0D0E0D082D083A380E722E4F5F078FB12004309
:20046E00F608A6F022746D75F065C0E0C0F0E52075F000C0E0C0F074021260B4158115813B
:20048E0015811581748875F065C0E0C0F0E50F75F000C0E0C0F0E510C0E0C0F0E51175F0C3
:2004AE0000C0E0C0F0E512C0E0C0F0740575F0001260B47FF612004F74BB75F065C0E0C064
:2004CE00F0E50B75F000C0E0C0F0E50CC0E0C0F0E50D75F000C0E0C0F0E50EC0E0C0F074DA
:2004EE000575F0001260B47FF612004FE4F50EF512227FFD7EFF1201E8E4F5F07F00120129
:20050E00CCF0A3C5F0F0C5F078FB120043E60886F012013418F608A6F012012645F0602205
:20052E00181818860108860289828A8312007089828A83E0120087C0E0C0F01261AD15811D
:20054E00158145F0700302060C7F001201CCE0A3F5F0E0C5F07B047C001201067F0012013A
:20056E00CCF0A3C5F0F0C5F078F9120043860108860289828A8312007089828A83E0120033
:20058E0087C0E0C0F01261BC158115817F021201CCF07F021201CCE01200877B3912007EAE
:2005AE00120153600B7F021201CCE0C39430800B7F021201CCE0C39441240A75F0007F0020
:2005CE001201CC1200692BC5F03CC5F07F001201CCF0A3C5F0F0C5F078F912004386010842
:2005EE00860289828A83E0A3F5F0E0C5F012012689828A83F0A3C5F0F0C5F00205167F0076
:20060E001201CCE0A3F5F0E0C5F07F030201E67FF17EFF1201E87F021201DAE98AF0C0E02C
:20062E00C0F0E4C0E0C0E0740A75F000C0E0C0F01261EE7FFA12004F7F021201DAE98AF099
:20064E007F0C1201CCF0A3C5F0F0C5F074097F0E1201CCF078FB1200438601088602898272
:20066E008A8312007089828A83E0120087C0E0C0F01261741581158145F0602E78FB1200A1
:20068E0043860108860289828A8312007089828A83E0120087C0E0C0F01261A81581158130
:2006AE0045F060067F0E1201CCE0700302072C7F0C1201CCE0A3F5F0E0C5F01201267F0C72
:2006CE001201CCF0A3C5F0F0C5F0120134F9AAF0C001C00278F912004386010886028982FB
:2006EE008A8312007089828A83E0D083D082F018860108860289828A83E0A3F5F0E0C5F08C
:20070E0012012689828A83F0A3C5F0F0C5F07F0E1201CCE0147F0E1201CCF00206627F02E6
:20072E001201DAE98AF0C0E0C0F0126211158115817F001201CCF0A3C5F0F0C5F07F0F027F
:20074E0001E67FFE7EFF1201E8E4F5F07F001201CCF0A3C5F0F0C5F07F001201CCE0A3F5C5
:20076E00F0E0C5F012014745F0601B78FB120043E60886F012013418F608A6F01201267B09
:20078E00007C0012015B45F070030207F678F7120043E60886F012012618F608A6F012019A
:2007AE0034F9AAF089828A83E0120087C0E0C0F008E60886F012012618F608A6F0120134EB
:2007CE00F9AAF089828A83E0120087FBACF0D0F0D0E0C39BC5F09CC5F07F001201CCF0A38B
:2007EE00C5F0F0C5F00207667F001201CCE0A3F5F0E0C5F07F020201E67FFF7EFF1201E867
:20080E00E47F001201CCF07F001201CCE075F0007B107C0012018070120208767F001201C7
:20082E00CCE0047F001201CCF080DC78FB120043E60886F07F001201CC1200652BC5F0343B
:20084E0000C5F0F9AAF07F001201CCE0C001C00279567A8412008712007789828A83E0F4A6
:20086E00D083D082F002082A740190847AF07F010201E67FFF7EFF1201E8E4F521E4F5F08C
:20088E009082BEF0A3C5F0F0C5F0E49082BDF074F475F081C0E0C0F0E4C0E0C0E074C97576
:2008AE00F000C0E0C0F01261EE7FFA12004FE4F5F0908389F0A3C5F0F0C5F074C075F08242
:2008CE00C0E0C0F0E4C0E0C0E074C975F000C0E0C0F01261EE7FFA12004FE4908455F074B8
:2008EE008C75F083C0E0C0F0E4C0E0C0E074C975F000C0E0C0F01261EE7FFA12004F740160
:20090E0090847AF0E47F001201CCF07F001201CCE075F0007B107C0012017A7012020987CE
:20092E007F001201CCE0047F001201CCF080DC7F001201CCE079567A841200871200777F11
:20094E00001201CCE0C001C00279687A8412008712007789828A83E0F4120087D083D0821C
:20096E0012006512007E1201717003020984E490847AF002098702092E90847AE0600302DC
:20098E0009CC745675F084C0E0C0F0E4C0E0C0E0741275F000C0E0C0F01261EE7FFA120026
:2009AE004F745675F084C0E0C0F0746675F065C0E0C0F012625A1581158115811581121794
:2009CE00491217E3746875F084C0E0C0F0120807158115817F010201E612038778FB1200C8
:2009EE0043E60886F090838BF0C209C2B490838BE075F000900A25020090E490838BF0D2FB
:200A0E0008C202E49095ADF0020A39C208D202E49095ADF0020A39190A0300190A02001924
:200A2E000A01000D0A00000000080A227FFB7EFF1201E878F9120043E60886F07F031201A1
:200A4E00CCF0A3C5F0F0C5F008E60886F07F011201CCF0A3C5F0F0C5F07F011201DAE98A37
:200A6E00F0C0E0C0F0740275F000C0E0C0F012050015811581158115817F001201CCF078C8
:200A8E00FB120043E60886F0C0E0C0F0743075F000C0E0C0F07402C0E0C0F01261EE7FFA4B
:200AAE0012004F7F031201CC12007089828A83E07003020AFD7F031201CC1200707F0012FC
:200ACE0001CCE089828A831200652B7F001201CCF07F031201CCE0A3F5F0E0C5F0120126BC
:200AEE007F031201CCF0A3C5F0F0C5F0020AB17F001201CCE0F4047F001201CCF078FB12D4
:200B0E00004386010886027F001201CCE075F0007B047C00120114C001C00290656B1200B3
:200B2E007012007789828A83E0D083D082F078FB120043E60886F02401C5F03400C5F0F939
:200B4E00AAF07F001201CCE0540FC001C00290656B12007012008712007789828A83E0D0FD
:200B6E0083D082F07F001201CCE012008754FFC5F05400C5F07F050201E6908455E06003A1
:200B8E00020C2E748C75F083C0E0C0F0E4C0E0C0E074C975F000C0E0C0F01261EE7FFA12D1
:200BAE00004F90838BE075F0007B007C001201887003020C1A798C7A83742489828A83F026
:200BCE00E4A20992E0F51F748C75F083C0E0C0F0E51F600774FF75F0658005740375F0664B
:200BEE00C0E0C0F012624A1581158115811581748C75F083C0E0C0F0745675F084C0E0C036
:200C0E00F012624A1581158115811581748C75F083C0E0C0F012628815811581908455F007
:200C2E0078FB120043E60886F07B0A7C00120169700C18E60886F07BFF7C0012016945F05E
:200C4E007003020CBFE4A20992E0F51F7003020C82748C75F083C0E0C0F0748C75F08324EA
:200C6E0001C5F03400C0F0C0E0120A3A1581158115811581748C75F083C0E0C0F0120442EE
:200C8E001581158178FB120043E60886F07B0A7C001201697003020CB7740A75F000C0E0B6
:200CAE00C0F01202D415811581E4908455F0020CEB748C75F0839084551200652BC5F03450
:200CCE0000C5F0F9AAF078FB120043E60886F089828A83F0908455E004908455F02278FB4F
:200CEE00120043860108860289828A83E07003020D2D18860108860289828A83E012008713
:200D0E00C0E0C0F0120B881581158178FB120043E60886F012012618F608A6F0020CEC2277
:200D2E007FFA7EFF1201E8E4F5F07F021201CCF0A3C5F0F0C5F078FB120043E60886F07FF3
:200D4E00001201CCF0A3C5F0F0C5F0E47F041201CCF07F041201CCE075F0007B027C0012D1
:200D6E00017A7003020FAE7F041201CCE075F000900F84020090C2097F001201CCE0A3F5BB
:200D8E00F0E0C5F01201267F001201CCF0A3C5F0F0C5F0120134F9AAF089828A83E0120058
:200DAE0087900EFB0200907F001201CC12007089828A83E01200877B2012007E12016970EB
:200DCE0003020DDD74017F041201CCF0020DE574037F041201CCF0020F0778FB120043E6CC
:200DEE000886F0C0E0C0F018E60886F02401C5F03400C0F0C0E0120A3A1581158115811510
:200E0E00817F051201CCF07F051201CCE07003020E9B74037F041201CCF0742F75F075C089
:200E2E00E0C0F09082BEE0A3F5F0E0C5F01201269082BEF0A3C5F0F0C0F0C0E01262CF155E
:200E4E00811581158115819082BEF0A3C5F0F0C5F090838BE075F0007B027C0012016970BC
:200E6E0003020E98740575F066C0E0C0F07F051201CCE075F000C0E0C0F0740275F0001240
:200E8E0060B41581158115811581020EED7F001201CCE0A3F5F0E0C5F02402C5F03400C5AC
:200EAE00F07F001201CCF0A3C5F0F0C5F07F001201CC12007089828A83E01200877B2012CB
:200ECE00007E1201697003020EE574017F041201CCF0D209020EED74037F041201CCF00238
:200EEE000F0774037F041201CCF0020F07E80D2300B50D21000000F00E020F90745675F024
:200F0E0084C0E0C0F07F001201CCE0A3F5F0E0C0F0C0E0745675F084C0E0C0F012628815E5
:200F2E00811581C0E0C0F01207507FFA12004F45F07003020F4F74037F041201CCF0020F17
:200F4E008174027F041201CCF0745675F084C0E0C0F0126288158115817F001201CC12009F
:200F6E00692BC5F03CC5F07F021201CCF0A3C5F0F0C5F0020F900A0F0100840D0000000090
:200F8E00900F7F001201CCE0A3F5F0E0C5F01201267F001201CCF0A3C5F0F0C5F0020D6056
:200FAE007F021201CCE0A3F5F0E0C5F07F060201E67FFD7EFF1201E8E4F5F07F011201CC3C
:200FCE00F0A3C5F0F0C5F012034545F070030212621203BC7F001201CCF0E4A20892E0F58A
:200FEE001F70030210087F001201CCE0120087C0E0C0F01202D4158115819082BDE06003EA
:20100E0002103074F475F081C0E0C0F0E4C0E0C0E074C975F000C0E0C0F01261EE7FFA12E0
:20102E00004F7F001201CCE01200879010A80200909082BDE070030210619082BDE01490BA
:20104E0082BDF079F47A81120087120077E489828A83F00210B40210B474F475F0819082F1
:20106E00BD1200652BC5F03400C5F0F9AAF07F001201CCE089828A83F09082BDE0049082C7
:20108E00BDF075F0007BC87C0012019070030210A574C79082BDF00210B464100A003F1017
:2010AE000800000067107F001201CCE01200877B0A12007E120169700302126290838BE0D4
:2010CE0075F00090124902009079F47A8189828A83E01200877B2A12007E120171700302F9
:2010EE00110174F475F0817F011201CCF0A3C5F0F0C5F002125D74F475F081C0E0C0F01215
:20110E000D2E158115817F011201CCF0A3C5F0F0C5F002125D9082BDE070030211A079F45B
:20112E007A8189828A83E01200879011900200900211A0741C75F066C0E0C0F01204421587
:20114E0081158174F475F081C0E0C0F012044215811581741E75F066C0E0C0F0120442152E
:20116E0081158174F475F081C0E0C0F0120D2E158115817F011201CCF0A3C5F0F0C5F002E5
:20118E0011A03E112D003E112A003E1124000000411102125D9082BDE0700302123379F48F
:2011AE007A8189828A83E012008790122302009002123374F475F081C0E0C0F0120D2E15F7
:2011CE008115817F011201CCF0A3C5F0F0C5F07F011201CCE0A3F5F0E0C5F045F070030298
:2011EE001220742075F066C0E0C0F012044215811581745675F084C0E0C0F012044215818B
:20120E001581742475F066C0E0C0F012044215811581021233BE112D00BE112A00BE1124C4
:20122E00000000C11102125D740175F000C0E0C0F01209E71581158102125DA311030023BA
:20124E0011020004110100D710000000003612E49082BDF07F011201CCE0A3F5F0E0C5F029
:20126E007F030201E690838BE075F0007B007C00120169700E90838BE075F0007B027C0045
:20128E0012016945F070030212AC78FB120043E60886F0C0E0C0F0120CEC158115812290F8
:2012AE00838BE075F0007B007C0012016970030212E0745675F084C0E0C0F0120442158102
:2012CE001581742875F066C0E0C0F012044215811581227FFD7EFF1201E878FB120043E66B
:2012EE000886F02401C5F03400C5F0F9AAF089828A83E01200877B3D12007E120169700344
:20130E0002143C18E60886F02402C5F03400C5F07F001201CCF0A3C5F0F0C5F07F00120150
:20132E00CCE0A3F5F0E0C0F0C0E0126288158115817B017C001201637003021429745675B4
:20134E00F084C0E0C0F0E4C0E0C0E0741275F000C0E0C0F01261EE7FFA12004FE47F0212AA
:20136E0001CCF07F021201CCE075F0007B107C0012017A600D7F001201CC12007089828A87
:20138E0083E070120213E67F021201CCE0047F021201CCF080CD7F021201CCE079567A8471
:2013AE001200871200777F001201CCE0A3F5F0E0C5F01201267F001201CCF0A3C5F0F0C50E
:2013CE00F0120134C001C002F9AAF089828A83E0D083D082F0021395745675F084C0E0C068
:2013EE00F0745675F084C0E0C0F012628815811581D004D0032BC5F03CC5F0F9AAF0742025
:20140E0089828A83F0121749746875F084C0E0C0F012080715811581021439742A75F0662A
:20142E00C0E0C0F012127315811581021487121749746875F084C0E0C0F01208071581159B
:20144E008174C075F082C0E0C0F0744475F066C0E0C0F0745675F084C0E0C0F0740375F0E0
:20146E00001260C57FFA12004F74C075F082C0E0C0F0120CEC158115817F030201E678FBCE
:20148E00120043E60886F018F608A6F074C075F082C0E0C0F0745775F066C0E0C0F07456BE
:2014AE0075F084C0E0C0F0740375F0001260C57FFA12004F74C075F082C0E0C0F0120CEC83
:2014CE0015811581788018E660FC881F74C075F082C0E0C0F0746875F066C0E0C0F0E51F73
:2014EE0075F000C0E0C0F0747FC0E0C0F0740475F0001260C57FF812004F74C075F082C01F
:20150E00E0C0F0120CEC158115812278FB120043E60886F018F608A6F074C075F082C0E042
:20152E00C0F0748275F066C0E0C0F0E50A75F000C0E0C0F09082BEE0A3F5F0E0C0F0C0E0D0
:20154E00740475F0001260C57FF812004F74C075F082C0E0C0F0120CEC15811581E4F50A0D
:20156E00E4F5F09082BEF0A3C5F0F0C5F0227FFE7EFF1201E878FB120043E60886F024016F
:20158E00C5F03400C5F07F001201CCF0A3C5F0F0C5F07F001201CC12007089828A83E0126A
:2015AE000087C0E0C0F01261A81581158145F070030215DE7F001201CCE0A3F5F0E0C0F00C
:2015CE00C0E0126211158115819095ADF002161874C075F082C0E0C0F074B175F066C0E0BF
:2015EE00C0F09095ADE075F000C0E0C0F0740375F0001260C57FFA12004F74C075F082C0FE
:20160E00E0C0F0120CEC158115817F020201E67FFE7EFF1201E878FB120043E60886F02447
:20162E0001C5F03400C5F07F001201CCF0A3C5F0F0C5F07F001201CC12007089828A83E0DA
:20164E001200879016EC02009074C075F082C0E0C0F074C575F066C0E0C0F090838BE0750D
:20166E00F000C0E0C0F0740375F0001260C57FFA12004F74C075F082C0E0C0F0120CEC15A5
:20168E008115810216F47F001201CC12007089828A83E0120087C0E0C0F01261A815811592
:2016AE008145F070030216D97F001201CCE0A3F5F0E0C0F0C0E012621115811581C0E0C0FB
:2016CE00F01209E7158115810216E974D575F066C0E0C0F0121273158115810216F457163D
:2016EE000000000094167F020201E690838BE075F0007B007C00120169700302174874C06A
:20170E0075F082C0E0C0F074ED75F066C0E0C0F078F7120043E60886F0C0E0C0F0740375A4
:20172E00F0001260C57FFA12004F74C075F082C0E0C0F012127315811581227FFD7EFF123F
:20174E0001E8E590F4540E1200877B0112007E1201147F001201CCF07F001201CCE04430FB
:20176E007F011201CCF0745675F084C0E0C0F0126288158115817F021201CCF07F021201FD
:20178E00CCE075F0007B027C0012019070030217C07F021201CCE0C3940279567A841200CA
:2017AE00871200777F011201CCE089828A83F00217D5E4F5F079567A841200777F01120124
:2017CE00CCE089828A83F07F001201CCE01200877F030201E6D290E4A29092E0F51F700394
:2017EE00021804740175F000C0E0C0F01209E715811581021810E4C0E0C0E01209E715817F
:20180E001581227FFA7EFF1201E878FB120043E60886F07F021201CCF0A3C5F0F0C5F07F19
:20182E00001201CCF0A3C5F0F0C5F07F001201CC12007089828A83E070030218EB7F0012ED
:20184E0001CC12007089828A83E01200877B2012007E12016970030218867F001201CCE0A2
:20186E00A3F5F0E0C5F01201267F001201CCF0A3C5F0F0C5F00218E87F021201CC120070D5
:20188E00C001C0027F001201CC12007089828A83E0120087C0E0C0F01261BC15811581D0CB
:2018AE0083D082F07F001201CCE0A3F5F0E0C5F01201267F001201CCF0A3C5F0F0C5F07FF7
:2018CE00021201CCE0A3F5F0E0C5F01201267F021201CCF0A3C5F0F0C5F00218397F0212B0
:2018EE0001CC120070E489828A83F078FB120043E60886F02401C5F03400C5F07F0012011E
:20190E00CCF0A3C5F0F0C5F018860108860289828A83E012008790238E02009078FB1200E8
:20192E0043E60886F0C0E0C0F01212E1158115810223D67F001201CC12007089828A83E09E
:20194E00120087C0E0C0F01261A81581158145F0700302197F7F001201CCE0A3F5F0E0C0A1
:20196E00F0C0E01262111581158190850AF00219B974C075F082C0E0C0F0740875F067C0C2
:20198E00E0C0F090850AE075F000C0E0C0F0740375F0001260C57FFA12004F74C075F082ED
:2019AE00C0E0C0F0120CEC158115810223D67F001201CC12007089828A83E0120087901A7D
:2019CE003B0200907F001201CCE0A3F5F0E0C5F02401C5F03400C0F0C0E012621115811543
:2019EE0081C0E0C0F012355515811581021A477F001201CCE0A3F5F0E0C5F02401C5F03474
:201A0E0000C0F0C0E012621115811581C0E0C0F012325D15811581021A47742A75F067C00D
:201A2E00E0C0F012127315811581021A47FD195400D21952000000281A0223D612148C123A
:201A4E002F35125E3512424D0223D678FB120043E60886F0C0E0C0F01215191581158102E9
:201A6E0023D67F001201CCE0A3F5F0E0C5F01201267F001201CCF0A3C5F0F0C5F012013439
:201A8E00F9AAF089828A83E0120087901BB60200907F001201CC12007089828A83E0120037
:201AAE0087C0E0C0F01261AD1581158145F060227F001201DAE98AF0C0E0C0F0740475F042
:201ACE0000C0E0C0F01205001581158115811581800A90655EE0A3F5F0E0C5F07F041201C9
:201AEE00CCF0A3C5F0F0C5F090655AE0A3F5F0E0C0F0C0E07F041201CCE0A3F5F0E0C0F0DE
:201B0E00C0E012496D1581158115811581021BC67F001201CC12007089828A83E0120087A3
:201B2E00C0E0C0F01261AD1581158145F060227F001201DAE98AF0C0E0C0F0740475F00048
:201B4E00C0E0C0F01205001581158115811581800A90655EE0A3F5F0E0C5F07F041201CC7C
:201B6E00F0A3C5F0F0C5F090655EE0A3F5F0E0C0F0C0E07F041201CCE0A3F5F0E0C0F0C065
:201B8E00E012496D1581158115811581021BC6124F17021BC6744575F067C0E0C0F0121200
:201BAE007315811581021BC69D1B52001E1B45009F1A44000000A31B0223D67F001201CCF9
:201BCE0012007089828A83E0120087C0E0C0F01261A81581158145F07003021C637F001293
:201BEE0001CCE0A3F5F0E0C0F0C0E0126211158115819095A7F0A3C5F0F0C5F07B147C00FD
:201C0E0012017A7003021C60741475F0009095A7F0A3C5F0F0C5F074C075F082C0E0C0F027
:201C2E00745E75F067C0E0C0F09095A7E0A3F5F0E0C0F0C0E0740375F0001260C57FFA12A6
:201C4E00004F74C075F082C0E0C0F012127315811581021C9E74C075F082C0E0C0F07487D7
:201C6E0075F067C0E0C0F09095A7E0A3F5F0E0C0F0C0E0740375F0001260C57FFA12004FE9
:201C8E0074C075F082C0E0C0F0120CEC158115810223D678FB120043E60886F0C0E0C0F01E
:201CAE0012157C158115810223D678FB120043E60886F0C0E0C0F012161D1581158102233A
:201CCE00D67F001201CCE0A3F5F0E0C5F02402C5F03400C5F0F9AAF089828A83E0120087DD
:201CEE00C39430C5F09400C5F07F041201CCF0A3C5F0F0C5F07F001201CCE0A3F5F0E0C597
:201D0E00F02401C5F03400C5F0F9AAF089828A83E01200877B3D12007E12016960287F040F
:201D2E001201CCE0A3F5F0E0C5F07B007C0012016360137F041201CCE0A3F5F0E0C5F07BFF
:201D4E00017C0012015345F07003021DEE7F001201CC12007089828A83E0120087901DDBE4
:201D6E000200907F041201CCE0A3F5F0E0C5F045F07003021D89D296021D8BC296021DEBA0
:201D8E007F041201CCE0A3F5F0E0C5F045F07003021DA6D295021DA8C295021DEB7F041245
:201DAE0001CCE0A3F5F0E0C5F045F07003021DC3D294021DC5C294021DEB74AB75F067C06C
:201DCE00E0C0F012127315811581021DEBAB1D43008E1D4200711D41000000C81D021DFECF
:201DEE0074C475F067C0E0C0F0121273158115810223D67F001201CC12007089828A83E0EB
:201E0E00120087C0E0C0F01261A81581158145F07003021E527F001201CCE0A3F5F0E0C004
:201E2E00F0C0E0126211158115819095ABF0A3C5F0F0C5F0E4F5F09095A9F0A3C5F0F0C502
:201E4E00F0021E8D74C075F082C0E0C0F074DD75F067C0E0C0F09095ABE0A3F5F0E0C0F037
:201E6E00C0E0740375F0001260C57FFA12004F74C075F082C0E0C0F0120CEC158115810224
:201E8E0023D67F001201CC12007089828A83E07003021FC67F001201CCE0A3F5F0E0C0F0B3
:201EAE00C0E0742D75F000C0E0C0F012631615811581158115817F021201CCF0A3C5F0F0A3
:201ECE00C5F07F021201CCE0A3F5F0E0C5F07B007C001201697003021F687F001201CC1203
:201EEE00007089828A83E0120087C0E0C0F01261A81581158145F07003021F557F0012018C
:201F0E00CCE0A3F5F0E0C0F0C0E0126211158115817F041201CCF0A3C5F0F0C5F07F0412BA
:201F2E0001CCE0A3F5F0E0C0F0C0E07F041201CCE0A3F5F0E0C0F0C0E0122C961581158134
:201F4E0015811581021F6574F575F067C0E0C0F012127315811581021FC37F001201CCE057
:201F6E00A3F5F0E0C0F0C0E0126211158115817F041201CCF0A3C5F0F0C5F07F041201CC39
:201F8E00E0A3F5F0E0C0F0C0E07F021201CCE0A3F5F0E0C5F02401C5F03400C0F0C0E012CE
:201FAE00621115811581C0E0C0F0122C961581158115811581021FDFE4C0E0C0E074FF75EC
:201FCE00F001C0E0C0F0122C9615811581158115810223D67F001201CCE0A3F5F0E0C0F035
:201FEE00C0E0740C75F068C0E0C0F0126333158115811581158145F0700302201E741175B4
:20200E00F068C0E0C0F0121273158115810220241203870200000223D67F001201CC1200F8
:20202E007089828A83E0120087C0E0C0F01261A81581158145F0700302206C7F001201CC66
:20204E00E0A3F5F0E0C0F0C0E012621115811581C0E0C0F0122AFB158115810220C47F0011
:20206E001201CC12007089828A83E01200877B4D12007E12016970030220B47F001201CCE5
:20208E00E0A3F5F0E0C5F02401C5F03400C0F0C0E012621115811581C0E0C0F012579F15B9
:2020AE008115810220C4742675F068C0E0C0F0121273158115810223D67F001201CC120030
:2020CE007089828A83E0120087C0E0C0F01261A81581158145F0700302210C7F001201CC25
:2020EE00E0A3F5F0E0C0F0C0E012621115811581C0E0C0F01259DF158115810221CE7F0053
:20210E001201CC12007089828A83E01200879021C20200907F001201CCE0A3F5F0E0C5F05F
:20212E001201267F001201CCF0A3C5F0F0C5F0F9AAF089828A83E0120087C0E0C0F0126126
:20214E00A81581158145F070030221717F001201CCE0A3F5F0E0C0F0C0E01262111581153B
:20216E0081F51C74C075F082C0E0C0F0743D75F068C0E0C0F0E51C75F000C0E0C0F0740359
:20218E001260C57FFA12004F74C075F082C0E0C0F0120CEC158115810221CE123EF102212A
:2021AE00CE746175F068C0E0C0F0121273158115810221CEA9215800222144000000AF2124
:2021CE000223D60223D6748175F068C0E0C0F0120CEC1581158174B675F068C0E0C0F0125A
:2021EE000CEC1581158174D175F068C0E0C0F0120CEC1581158174F275F068C0E0C0F01280
:20220E000CEC15811581741D75F069C0E0C0F0120CEC15811581745675F069C0E0C0F012AD
:20222E000CEC15811581748F75F069C0E0C0F0120CEC1581158174C975F069C0E0C0F012A8
:20224E000CEC1581158174F175F069C0E0C0F0120CEC15811581741975F06AC0E0C0F012D5
:20226E000CEC15811581745175F06AC0E0C0F0120CEC15811581747475F06AC0E0C0F012F9
:20228E000CEC1581158174A375F06AC0E0C0F0120CEC1581158174CF75F06AC0E0C0F0122C
:2022AE000CEC1581158174ED75F06AC0E0C0F0120CEC15811581741775F06BC0E0C0F01279
:2022CE000CEC15811581744F75F06BC0E0C0F0120CEC15811581747E75F06BC0E0C0F0128F
:2022EE000CEC1581158174AD75F06BC0E0C0F0120CEC1581158174E075F06BC0E0C0F012AF
:20230E000CEC15811581740875F06CC0E0C0F0120CEC15811581744575F06CC0E0C0F012CC
:20232E000CEC15811581748175F06CC0E0C0F0120CEC1581158174B575F06CC0E0C0F012C3
:20234E000CEC1581158174DB75F06CC0E0C0F0120CEC1581158174FA75F06CC0E0C0F01204
:20236E000CEC158115810223D678FB120043E60886F0C0E0C0F01216F9158115810223D66C
:20238E00D4213F00D1210000C720540027205300E21F5200901E5100011E5000CF1C4F0039
:2023AE00B81C4E00A11C4C00C91B4900701A4800591A45004A1A4400BC19430041194200D1
:2023CE002A194100000077237F060201E6C2B3E4F522E4F514E4F517747B75F0EDF5188543
:2023EE00F019E4F51AE4F531742890850AF0747B75F084C0E0C0F0E4C0E0C0E0742075F0D9
:20240E0000C0E0C0F01261EE7FFA12004FE4F528F527F526F525749B75F084C0E0C0F0E4A5
:20242E00C0E0C0E0742075F000C0E0C0F01261EE7FFA12004FE4F52CF52BF52AF529E4F58F
:20244E0016F51574BB75F084C0E0C0F0E4C0E0C0E0744F75F000C0E0C0F01261EE7FFA125E
:20246E00004F740B75F085C0E0C0F0E4C0E0C0E0E475F004C0E0C0F01261EE7FFA12004F4A
:20248E00E58854CFF588E58954F0F5894401F589E4F58AF58CD2B9D2A9D28CD288D2A822F0
:2024AE00C0E0C0D0C28C85188A85198CD28CA2149215A2B2B39214C0F0C083C082C000E5FD
:2024CE0014B4020280044002740075F003A49024E0730224E9022528022570051AE531604B
:2024EE00021531E5324533600DC3E5329401F532E5339400F5332016030226F3C21675146B
:20250E0001751A007515007518BC7519FDC28C85188A85198CD28C0226F39084BBE51525B9
:20252E0082F582E5833400F583E0A2E092B30515E515B5160050030226F3C2B37514007519
:20254E00187B7519EDC28C85188A85198CD28CE51675F00884251AF51A90850AE0F5310201
:20256E0026F3301305C2130226F3E517B40A0280044002740A75F003A490258B730225AC6A
:20258E000225C90225DC0225FD02260A0226330226410226540226750226820226EA301407
:2025AE006D7518BC7519FDC28CE518241EF58AE43519F58CD28C0517022617A215B0145089
:2025CE004D752D00752E007515090517803BA215B01492D5A214B01572D55032E52EA21402
:2025EE0013F52EE52D13F52DD5151E0517801AA215B01450197515020517800D20150F2015
:20260E00140CD5150405178000D2130226F375170A0226F375140075170075187B7519EDB9
:20262E00B2970226F3A215B3821450E2751509051780D6A215B01450D5752F007530007593
:20264E001509051780C3A215B01492D5A214B01572D550BAE530A21413F530E52F13F52FF3
:20266E00D515A6051780A2A215B01450A175150305178071201497D5156BE52D652F7094AE
:20268E00E52E6530708E852E83852D8275F007C3E58313F583E58213F582D5F0F385832E1B
:2026AE0085822DE52925E0249BF58274843400F583E52DF0A3E52EF005297410B529028031
:2026CE00025003752900052BE52BB52C0280044002F52C7406251AF51A0226222015062082
:2026EE001403022622E51AB4C2004006D217243EF51AD000D082D083D0F0D0D0D0E032227D
:20270E00C0E0C0F0C0D0C083C082E514B4020280044002740025E0902729738004801F8060
:20272E001F7518E17519FEC28C85188A85198CD28C751700751500751402B297800E800C71
:20274E00C28C758AE1758CFED28C8000D082D083D0D0D0F0D0E0322278F9120043E608861D
:20276E00F05401C5F05400C5F07B007C0012016970030227A9088601088602740189828A67
:20278E0083F018E60886F02401C5F03400C5F0F9AAF0E489828A83F00227D078FB12004339
:2027AE008601088602E489828A83F018E60886F02401C5F03400C5F0F9AAF0740189828A2C
:2027CE0083F0227FFF7EFF1201E8740175F000C0E0C0F078F9120043E60886F02400C5F033
:2027EE003400C0F0C0E01227661581158115811581E4C0E0C0E078F9120043E60886F024DE
:20280E0002C5F03400C0F0C0E0122766158115811581158178FB120043E60886F02404C55F
:20282E00F03400C5F018F608A6F0E47F001201CCF07F001201CCE075F0007B097C0012011D
:20284E007A70120228AE7F001201CCE0047F001201CCF080DC78F9120043E60886F0C0E0E0
:20286E00C0F008E60886F0C0E0C0F0122766158115811581158178F9120043E60886F07B42
:20288E00017C0012011418F608A6F008E60886F02402C5F03400C5F018F608A6F002285480
:2028AE00E4C0E0C0E078F9120043E60886F0C0E0C0F012276615811581158115817F0102F3
:2028CE0001E678FB120043E60886F07BFF7CFF12017160069095ADE05402700302293274AC
:2028EE00C075F082C0E0C0F0741675F06DC0E0C0F078F7120043E60886F0C0E0C0F018E6B1
:20290E000886F0C0E0C0F0740475F0001260C57FF812004F74C075F082C0E0C0F0120CEC7A
:20292E001581158174BB75F084C0E0C0F0E4C0E0C0E0744F75F000C0E0C0F01261EE7FFA7F
:20294E0012004F78FB120043E60886F0C0E0C0F074BB75F0842418C5F03400C0F0C0E012ED
:20296E0027D1158115811581158178FB120043E60886F0C0E0C0F074BB75F0842434C5F058
:20298E003400C0F0C0E01227D11581158115811581744FF516D216227FFE7EFF1201E8E591
:2029AE002B70030229FBE52A75F000C333C5F033C5F0799B7A8412007789828A83E0A3F513
:2029CE00F0E0C5F07F001201CCF0A3C5F0F0C5F0152B052AE52AE52A75F0007B107C00120E
:2029EE00019070030229F8E4F52A022A0B74FFF5F07F001201CCF0A3C5F0F0C5F07F001234
:202A0E0001CCE0A3F5F0E0C5F07BFF7CFF12017160069095ADE054017003022A7674C0753A
:202A2E00F082C0E0C0F0742975F06DC0E0C0F07F001201CCE0A3F5F0E0C0F0C0E07F001280
:202A4E0001CCE0A3F5F0E0C0F0C0E0740475F0001260C57FF812004F74C075F082C0E0C09C
:202A6E00F0120CEC158115817F001201CCE0A3F5F0E0C5F07F020201E67FFE7EFF1201E868
:202A8E001229A67F001201CCF0A3C5F0F0C5F07F001201CCE0A3F5F0E0C5F07BFF7CFF129A
:202AAE00017160137F001201CCE0A3F5F0E0C5F07BFF7C0112017A45F07003022AF67F00FB
:202ACE001201CCE0A3F5F0E0C5F0C333C5F033C5F0790B7A85120077740175F00089828AFE
:202AEE0083F0A3C5F0F0C5F07F020201E67FFE7EFF1201E878FB120043E60886F07BFF7CD7
:202B0E0001120180600CE52775F0007B107C0012017A45F07003022B91E52575F000C333D7
:202B2E00C5F033C5F0797B7A8412007778FB120043E60886F089828A83F0A3C5F0F0C5F03E
:202B4E000525E525E52575F0007B107C001201907003022B66E4F5250527E527E52775F06D
:202B6E0000AB287C001201887003022B7FE527F528E4F5F07F001201CCF0A3C5F0F0C5F001
:202B8E00022BA2740175F0007F001201CCF0A3C5F0F0C5F07F001201CCE0A3F5F0E0C5F0D8
:202BAE007F020201E67FFE7EFF1201E8E5277003022C08E52675F000C333C5F033C5F07977
:202BCE007B7A8412007789828A83E0A3F5F0E0C5F07F001201CCF0A3C5F0F0C5F015270544
:202BEE0026E526E52675F0007B107C001201907003022C05E4F526022C1874FFF5F07F00BA
:202C0E001201CCF0A3C5F0F0C5F07F001201CCE0A3F5F0E0C5F07F020201E67FFE7EFF1209
:202C2E0001E8E53112008712014745F0600CE51475F0007B007C0012016945F07003022C4C
:202C4E0091122BB37F001201CCF0A3C5F0F0C5F07F001201CCE0A3F5F0E0C5F07BFF7CFF4A
:202C6E001201717003022C8B7F001201CCE0A3F5F0E0C0F0C0E01228D01581158190850A4B
:202C8E00E0F5317F020201E67FFD7EFF1201E878F9120043E60886F0088603088604120162
:202CAE00697003022D4674C075F082C0E0C0F0743C75F06DC0E0C0F0181818E60886F0C00C
:202CCE00E0C0F018E60886F0C333C5F033C5F0790B7A8512007789828A83E0A3F5F0E0C516
:202CEE00F045F06007740175F0008003E4F5F0C0E0C0F0740475F0001260C57FF812004FD8
:202D0E0074C075F082C0E0C0F0120CEC1581158178F9120043E60886F0C333C5F033C5F047
:202D2E00790B7A85120077E4F5F089828A83F0A3C5F0F0C5F0022F3074C075F082C0E0C0CF
:202D4E00F0744675F06DC0E0C0F078F5120043E60886F0C0E0C0F008E60886F0C0E0C0F067
:202D6E00740475F0001260C57FF812004F74C075F082C0E0C0F0120CEC1581158178F91235
:202D8E000043E60886F00886030886041201537003022F20E47F001201CCF0181818E608C9
:202DAE0086F07F011201CCF0A3C5F0F0C5F078F9120043E60886F02408C5F03400C5F07FD0
:202DCE00011201CC12006912015B60157F011201CCE0A3F5F0E0C5F0088603088604120115
:202DEE005345F07020022E967F011201CCE0A3F5F0E0C5F01201267F011201CCF0A3C5F0AB
:202E0E00F0C5F080A97F001201CCE075F0007B017C001201147F001201CCF07F011201CC67
:202E2E00E0A3F5F0E0C5F0C333C5F033C5F0790B7A8512007789828A83E0A3F5F0E0C5F0D3
:202E4E0045F06007748075F0008003E4F5F07F001201CC1200654B7F001201CCF07F011223
:202E6E0001CCE0A3F5F0E0C5F0C333C5F033C5F0790B7A85120077E4F5F089828A83F0A367
:202E8E00C5F0F0C5F0022DF678F9120043E60886F02408C5F03400C5F07F011201CC120040
:202EAE0069C39BC5F09CC5F0FBACF07F001201CCE075F0001201147F001201CCF074C075DF
:202ECE00F082C0E0C0F0745275F06DC0E0C0F07F001201CCE075F000C0E0C0F0740375F06B
:202EEE00001260C57FFA12004F74C075F082C0E0C0F0120CEC1581158178F9120043E6085E
:202F0E0086F02408C5F03400C5F018F608A6F0022D8B740A75F000C0E0C0F0120B8815818F
:202F2E0015817F030201E6745775F06DC0E0C0F0120CEC1581158174C075F082C0E0C0F0F4
:202F4E00746D75F06DC0E0C0F0E51475F000C0E0C0F0E517C0E0C0F0E53175F000C0E0C08B
:202F6E00F090850AE075F000C0E0C0F0740675F0001260C57FF412004F74C075F082C0E0FA
:202F8E00C0F0120CEC1581158174C075F082C0E0C0F074A575F06DC0E0C0F0E51575F00038
:202FAE00C0E0C0F074031260C57FFA12004F74C075F082C0E0C0F0120CEC1581158174C056
:202FCE0075F082C0E0C0F074B375F06DC0E0C0F0E51675F000C0E0C0F0E522C0E0C0F0E577
:202FEE001A75F000C0E0C0F074051260C57FF612004F74C075F082C0E0C0F0120CEC158163
:20300E00158174C075F082C0E0C0F074DE75F06DC0E0C0F0E52575F000C0E0C0F0E526C0A3
:20302E00E0C0F0E52775F000C0E0C0F0E528C0E0C0F0740675F0001260C57FF412004F7476
:20304E00C075F082C0E0C0F0120CEC1581158174C075F082C0E0C0F0741275F06EC0E0C011
:20306E00F0E52575F000C333C5F033C5F0797B7A8412007789828A83E0A3F5F0E0C0F0C005
:20308E00E0740375F0001260C57FFA12004F74C075F082C0E0C0F0120CEC1581158174C080
:2030AE0075F082C0E0C0F0742575F06EC0E0C0F0E52675F000C333C5F033C5F0797B7A841A
:2030CE0012007789828A83E0A3F5F0E0C0F0C0E0740375F0001260C57FFA12004F74C07513
:2030EE00F082C0E0C0F0120CEC1581158174C075F082C0E0C0F0743775F06EC0E0C0F0E5AC
:20310E002975F000C0E0C0F0E52AC0E0C0F0E52B75F000C0E0C0F0E52CC0E0C0F07406754F
:20312E00F0001260C57FF412004F74C075F082C0E0C0F0120CEC1581158174C075F082C00A
:20314E00E0C0F0746B75F06EC0E0C0F0E52975F000C333C5F033C5F0799B7A8412007789A5
:20316E00828A83E0A3F5F0E0C0F0C0E0740375F0001260C57FFA12004F74C075F082C0E072
:20318E00C0F0120CEC1581158174C075F082C0E0C0F0747E75F06EC0E0C0F0E52A75F00047
:2031AE00C333C5F033C5F0799B7A8412007789828A83E0A3F5F0E0C0F0C0E0740375F00047
:2031CE001260C57FFA12004F74C075F082C0E0C0F0120CEC15811581740A75F000C0E0C0EC
:2031EE00F0120B8815811581E4F528F52C2290000075F014C2AFC297C28CC28D758C4C758A
:20320E008A00D28C108D0C30B5FA108D1620B5FAA380F1758C4C758A00B297209813D5F075
:20322E00E9800E758C4C758A00B297209803D5F0D38583F0E58290890BF0A3E5F0F0D297DD
:20324E00D28DD2AF90890BE0A3F5F0E0C5F0227FFC7EFF1201E878FB120043E60886F01806
:20326E00F608A6F0748F75F06EC0E0C0F0120CEC1581158174C075F082C0E0C0F074AE754E
:20328E00F06EC0E0C0F0747075F094C0E0C0F0747075F017C0E0C0F0746475F000C0E0C0F8
:2032AE00F074051260C57FF612004F74C075F082C0E0C0F0120CEC1581158174DB75F06EC7
:2032CE00C0E0C0F0120CEC158115811203871231FC7F001201CCF0A3C5F0F0C5F0120345DA
:2032EE0045F060030234CD74C075F082C0E0C0F074F975F06EC0E0C0F07F001201CCE0A349
:20330E00F5F0E0C0F0C0E0740375F0001260C57FFA12004F74C075F082C0E0C0F0120CEC28
:20332E00158115817F001201CCE0A3F5F0E0C5F07BB87C8812017A700302338574C075F06E
:20334E0082C0E0C0F0740275F06FC0E0C0F074B875F088C0E0C0F0740375F0001260C57FF8
:20336E00FA12004F74C075F082C0E0C0F0120CEC158115810234C37F001201CCE0A3F5F084
:20338E00E0C5F07B287CA012018870030233D874C075F082C0E0C0F0741175F06FC0E0C08C
:2033AE00F0742875F0A0C0E0C0F0740375F0001260C57FFA12004F74C075F082C0E0C0F0C6
:2033CE00120CEC158115810234C3748675F0887F021201CCF0A3C5F0F0C5F07F021201CC1C
:2033EE00E0A3F5F0E0C5F07B5A7CA012018070250234B37F021201CCE0A3F5F0E0C5F0243F
:20340E0064C5F03400C5F07F021201CCF0A3C5F0F0C5F080C67F001201CCE0A3F5F0E0C59E
:20342E00F07F021201CC120069120190601F7F021201CCE0A3F5F0E0C5F02464C5F03400C3
:20344E00C5F07F001201CC12006912019045F07003023475742A75F000C0E0C0F0120B88E2
:20346E00158115810234B07F021201CCE0A3F5F0E0C5F07B3E7C9412016970030234A074CD
:20348E007C75F000C0E0C0F0120B88158115810234B0742075F000C0E0C0F0120B881581B2
:2034AE001581023401741F75F06FC0E0C0F0120CEC1581158112034545F070030232D91223
:2034CE0003A9742275F06FC0E0C0F0120CEC158115817F040201E690890D7918C2AFC29755
:2034EE00C28CC28D758C00758A00D28C30B20C308DFAC28DB29720984980F1C28C758C00C5
:20350E00758A00D28CC28D208D3830B2FAE58C858AF0B58CF8B4030280D240D0C5F0F0A324
:20352E00E5F0F0A3208D1B20B2FAE58C858AF0B58CF8C5F0F0A3E5F0F0A3208D0530B2FA9A
:20354E00D9E2D297D2AF227FF57EFF1201E8744675F06FC0E0C0F0120CEC158115817474AE
:20356E0075F06FC0E0C0F0120CEC1581158174A075F06FC0E0C0F0120CEC15811581740DF4
:20358E0075F089C0E0C0F0E4C0E0C0E0743275F000C0E0C0F01261EE7FFA12004F12038789
:2035AE001234E512034545F06018E4F5F0790D7A8912007789828A83E0A3F5F0E0C5F012C9
:2035CE00014745F06003023EE974187F001201CCF07F001201CCE075F0007B017C0012014C
:2035EE0088701202367A7F001201CCE0147F001201CCF080DC7F001201CCE075F000C3336C
:20360E00C5F033C5F0790D7A891200777F001201CCE075F000C333C5F033C5F0C001C00234
:20362E00790D7A891200777F001201CCE0C3940175F000C333C5F033C5F0C001C002790DD3
:20364E007A89120077D083D082E0A3F5F0E0C5F089828A83120069C39BC5F09CC5F0D083E4
:20366E00D082F0A3C5F0F0C5F00235F4E47F001201CCF07F001201CCE075F0007B197C00ED
:20368E0012017A70120238AF7F001201CCE0047F001201CCF080DC78FB120043E60886F00C
:2036AE007B037C00120163700302373E74C075F082C0E0C0F074BE75F06FC0E0C0F07F0062
:2036CE001201CCE075F000C0E0C0F07F001201CCE075F000C333C5F033C5F0790D7A891297
:2036EE00007789828A83E0A3F5F0E0C0F0C0E07F001201CCE075F000C333C5F033C5F079E6
:20370E000D7A8912007789828A83E0A3F5F0E0C0F0C0E0740575F0001260C57FF612004F67
:20372E0074C075F082C0E0C0F0120CEC158115817F001201CCE075F000C333C5F033C5F0A4
:20374E00790D7A8912007789828A83E0A3F5F0E0C5F0C333C5F033C5F07F051201CCF0A3AB
:20376E00C5F0F0C5F07F051201CCE0A3F5F0E0C5F0240CC5F03400C5F07B197C001200D3BE
:20378E007F051201CCF0A3C5F0F0C5F07F001201CCE075F000C333C5F033C5F0790D7A890C
:2037AE0012007789828A83E0A3F5F0E0C5F02464C5F03400C5F07BC87C001200D37F0712FB
:2037CE0001CCF0A3C5F0F0C5F07F001201CCE075F000C333C5F033C5F0790D7A89120077D9
:2037EE007F051201CCE0A3F5F0E0C5F07F071201CC1200692BC5F03CC5F089828A83120080
:20380E00692BC5F03CC5F089828A83F0A3C5F0F0C5F078FB120043E60886F07B037C001223
:20382E00016370030238AC74C075F082C0E0C0F074D875F06FC0E0C0F07F001201CCE0752F
:20384E00F000C333C5F033C5F0790D7A8912007789828A83E0A3F5F0E0C0F0C0E07F001284
:20386E0001CCE075F000C333C5F033C5F0790D7A8912007789828A83E0A3F5F0E0C0F0C0B3
:20388E00E0740475F0001260C57FF812004F74C075F082C0E0C0F0120CEC15811581023675
:2038AE0096E4F5F0790D7A8912007789828A83E0A3F5F0E0C5F07B087C001200B97F051214
:2038CE0001CCF0A3C5F0F0C5F07F051201CCE0A3F5F0E0C5F07B0A7C001200D37F05120143
:2038EE00CCF0A3C5F0F0C5F078FB120043E60886F07B017C00120163700302396F74C075A1
:20390E00F082C0E0C0F074E975F06FC0E0C0F0E4F5F0790D7A8912007789828A83E0A3F5EB
:20392E00F0E0C0F0C0E07F051201CCE0A3F5F0E0C0F0C0E0740475F0001260C57FF81200C1
:20394E004F74C075F082C0E0C0F0120CEC15811581741375F070C0E0C0F0120CEC15811508
:20396E0081E4F5F0790D7A891200777F051201CCE0A3F5F0E0C5F089828A83F0A3C5F0F02D
:20398E00C5F0E47F021201CCF07F021201CCE075F0007B057C0012017A7012023AAE7F0215
:2039AE001201CCE0047F021201CCF080DC7F021201CCE075F000C333C5F033C5F079717AEE
:2039CE0089120077E4F5F0C001C002790D7A891200777F021201CCE0240175F000C333C5E4
:2039EE00F033C5F02401C5F03400C5F089828A831200691200B9D083D082F0A3C5F0F0C51E
:203A0E00F07F021201CCE075F000C333C5F033C5F079717A8912007789828A83E0A3F5F07A
:203A2E00E0C5F07B027C0012011489828A83F0A3C5F0F0C5F078FB120043E60886F07B0116
:203A4E007C001201637003023AAB74C075F082C0E0C0F0743075F070C0E0C0F07F02120144
:203A6E00CCE075F000C333C5F033C5F079717A8912007789828A83E0A3F5F0E0C0F0C0E06E
:203A8E00740375F0001260C57FFA12004F74C075F082C0E0C0F0120CEC158115810239ACA3
:203AAE0078FB120043E60886F07B017C001201637003023AD3743475F070C0E0C0F0120CF1
:203ACE00EC15811581E4F5F07F091201CCF0A3C5F0F0C5F0E47F011201CCF074017F00126A
:203AEE0001CCF07F001201CCE075F0007B197C0012017A60227F001201CCE075F000C333A0
:203B0E00C5F033C5F0790D7A8912007789828A83E0A3F5F0E0C5F045F07012023E7D7F00E0
:203B2E001201CCE0047F001201CCF080B678FB120043E60886F07B027C0012016370030220
:203B4E003BC774C075F082C0E0C0F0743875F070C0E0C0F07F001201CCE075F000C0E0C016
:203B6E00F07F001201CCE075F000C333C5F033C5F0790D7A8912007789828A83E0A3F5F07F
:203B8E00E0C0F0C0E0E4F5F079717A8912007789828A83E0A3F5F0E0C0F0C0E0740575F01A
:203BAE00001260C57FF612004F74C075F082C0E0C0F0120CEC158115817F001201CCE07596
:203BCE00F000C333C5F033C5F0790D7A89120077E4F5F0C001C00279717A89120077D0832D
:203BEE00D082E0A3F5F0E0C5F089828A831200691201807003023C7F7F001201CCE075F06F
:203C0E0000C333C5F033C5F0790D7A8912007789828A83E0A3F5F0E0C5F045F07003023CF6
:203C2E005778FB120043E60886F07B027C001201637003023C54744B75F070C0E0C0F01289
:203C4E000CEC15811581023C7C78FB120043E60886F07B027C001201637003023C7C745DDF
:203C6E0075F070C0E0C0F0120CEC15811581023B2C7F001201CCE075F000C333C5F033C52C
:203C8E00F0790D7A89120077740875F000C001C00279717A89120077D083D082E0A3F5F02D
:203CAE00E0C5F089828A831200691201887003023CE878FB120043E60886F07B027C001263
:203CCE0001637003023CE5746775F070C0E0C0F0120CEC15811581023B2C74017F02120134
:203CEE00CCF07F021201CCE075F0007B047C0012017A7012023E557F021201CCE0047F02F1
:203D0E001201CCF080DC7F001201CCE075F000C333C5F033C5F0790D7A891200777F02128F
:203D2E0001CCE075F000C333C5F033C5F0C001C00279717A89120077D083D082E0A3F5F0CA
:203D4E00E0C5F089828A831200691201807003023E527F001201CCE075F000C333C5F03314
:203D6E00C5F0790D7A8912007789828A83E0A3F5F0E0C5F0C333C5F033C5F07F031201CC65
:203D8E00F0A3C5F0F0C5F07F021201CCE02401FB7F031201CCE0A3F5F0E0C5F07C001200DC
:203DAE00D37F031201CCF0A3C5F0F0C5F078FB120043E60886F07B027C00120163700302C4
:203DCE003E1C74C075F082C0E0C0F0747D75F070C0E0C0F07F021201CCE0240175F000C070
:203DEE00E0C0F07F031201CCE0A3F5F0E0C0F0C0E0740475F0001260C57FF812004F74C00C
:203E0E0075F082C0E0C0F0120CEC158115817F091201CCE0A3F5F0E0C5F07F031201CC1250
:203E2E0000692BC5F03CC5F07F091201CCF0A3C5F0F0C5F07F011201CCE0047F011201CC44
:203E4E00F0023E55023D0578FB120043E60886F07B027C001201637003023E7A740A75F0E0
:203E6E0000C0E0C0F0120B8815811581023B2C7F091201CCE0A3F5F0E0C5F07F011201CCE7
:203E8E001200657C001200D37F091201CCF0A3C5F0F0C5F074C075F082C0E0C0F0749E75F6
:203EAE00F070C0E0C0F07F091201CCE0A3F5F0E0C0F0C0E0740375F0001260C57FFA1200A7
:203ECE004F74C075F082C0E0C0F0120CEC1581158112034545F0700302358C1203A97F0BD7
:203EEE000201E690655AE0A3F5F0E0C5F090959DF0A3C5F0F0C0F0C0E0E4C0E0C0E090651C
:203F0E005CE0A3F5F0E0C0F0C0E01261EE7FFA12004FE4F5F090959FF0A3C5F0F0C5F0E406
:203F2E00F5F09095A5F0A3C5F0F0C5F090959DE0A3F5F0E0C5F02402C5F03400C5F090952F
:203F4E00A1F0A3C5F0F0C5F09095A3F0A3C5F0F0C5F0E4F5F0F51D85F01E22E4F52474C847
:203F6E00F51C90655AE0A3F5F0E0C5F090959DF0A3C5F0F0C5F074E775F003C0E0C0F01202
:203F8E003FB4158115817B007C0012014D7003023FB374B875F070C0E0C0F01212731581B8
:203FAE001581123EF12278FB120043E60886F018F608A6F09095ADE05420700302401174C2
:203FCE00C075F082C0E0C0F074E675F070C0E0C0F090959DE0A3F5F0E0C0F0C0E018E608FD
:203FEE0086F0C0E0C0F0740475F0001260C57FF812004F74C075F082C0E0C0F0120CEC1577
:20400E00811581E4F5F09095A5F0A3C5F0F0C5F090959D12007089828A83E0A3F5F0E0C592
:20402E00F045F0600302404DE50A4440F50A74FFF5F09095A5F0A3C5F0F0C5F002422490E2
:20404E00959D12007089828A83E0A3F5F0E0C5F07BE77C03120188701490959D12007089BC
:20406E00828A83E0A3F5F0E0C5F012014745F07003024099E50A4440F50A74FFF5F09095DA
:20408E00A5F0A3C5F0F0C5F00242249095ADE0542070030240B7740A75F071C0E0C0F012D0
:2040AE000CEC1581158112424D90959DE0A3F5F0E0F58385F082E0A3FAE0A3FBC082C08334
:2040CE0090959FEAF0A3EBF0D083D082EA4B700D430A209095A5E4F0A3F0024224E582856D
:2040EE0083F0C082C0839095A1F0A3E5F0F0D083D082E0A3F51DE0A3F51EE0A3FEE0A3FFC9
:20410E00C082C0839095A5EEF0A3EFF0D083D082751B8979DF7C007D01B297EEC39DFEEF4E
:20412E009400FF50030241D6BC0040ED75F002A4FCADF0E0A3851BA0F309B90002051BE06B
:20414E00A3851BA0F309B90002051BE4851BA0F309B90002051BCC70011D14CCEC4D70D3E6
:20416E007C01E0A3FD70707C03806CBC013EED75F002A4FCADF0E0A3851BA0F309B90002E3
:20418E00051BE4851BA0F309B90002051B851BA0F309B90002051BCC70011D14CCEC4D70FC
:2041AE00D57C00E0A3FD702F7C02802BBC020B7C01E0A3FD70217C04801DBC030B7C00E0BE
:2041CE00A3FD70137C04800F9095A574FFF0A3F07C04430A40803FBC04005003024127EEA8
:2041EE004F70E5CA70011B14CAC082C0838583F0E5829095A3F0A3E5F0F0D083D08278FBBD
:20420E00120043E608B51D0280030240DAE6B51E0280030240DA9095ADE0542070030242A3
:20422E0042742975F071C0E0C0F0120CEC1581158112424D9095A5E0A3F5F0E0C5F0227F2C
:20424E00FA7EFF1201E8744775F071C0E0C0F0120CEC1581158174C075F082C0E0C0F074E8
:20426E005575F071C0E0C0F090959DE0A3F5F0E0C0F0C0E09095A1E0A3F5F0E0C0F0C0E0FD
:20428E009095A3E0A3F5F0E0C0F0C0E0740575F0001260C57FF612004F74C075F082C0E00A
:2042AE00C0F0120CEC1581158174C075F082C0E0C0F0747F75F071C0E0C0F090959FE0A33F
:2042CE00F5F0E0C0F0C0E0E51D851EF0C0E0C0F09095A5E0A3F5F0E0C0F0C0E0740575F096
:2042EE00001260C57FF612004F74C075F082C0E0C0F0120CEC1581158174A875F071C0E070
:20430E00C0F0120CEC15811581E4F5F07F001201CCF0A3C5F0F0C5F07F001201CCE0A3F5BF
:20432E00F0E0C5F07B007C0412014D70250246797F001201CCE0A3F5F0E0C5F02418C5F0ED
:20434E003400C5F07F001201CCF0A3C5F0F0C5F080C67F001201CCE0A3F5F0E0C5F079DF22
:20436E007A89120077E98AF07F041201CCF0A3C5F0F0C5F074C075F082C0E0C0F074B675E7
:20438E00F071C0E0C0F07F041201CCE0A3F5F0E0C5F02402C5F03400C5F0F9AAF089828A13
:2043AE0083E075F000C0E0C0F07F041201CCE0A3F5F0E0C5F02400C5F03400C5F0F9AAF023
:2043CE0089828A83E0A3F5F0E0C0F0C0E07F041201CCE0A3F5F0E0C5F02405C5F03400C5E9
:2043EE00F0F9AAF089828A83E075F000C0E0C0F07F041201CCE0A3F5F0E0C5F02403C5F044
:20440E003400C5F0F9AAF089828A83E0A3F5F0E0C0F0C0E0740675F0001260C57FF41200C7
:20442E004F74C075F082C0E0C0F0120CEC1581158174C075F082C0E0C0F074CA75F071C03F
:20444E00E0C0F07F041201CCE0A3F5F0E0C5F02408C5F03400C5F0F9AAF089828A83E07595
:20446E00F000C0E0C0F07F041201CCE0A3F5F0E0C5F02406C5F03400C5F0F9AAF089828A9F
:20448E0083E0A3F5F0E0C0F0C0E07F041201CCE0A3F5F0E0C5F0240BC5F03400C5F0F9AA24
:2044AE00F089828A83E075F000C0E0C0F07F041201CCE0A3F5F0E0C5F02409C5F03400C517
:2044CE00F0F9AAF089828A83E0A3F5F0E0C0F0C0E0740675F0001260C57FF412004F74C07D
:2044EE0075F082C0E0C0F0120CEC1581158174C075F082C0E0C0F074DE75F071C0E0C0F05E
:20450E007F041201CCE0A3F5F0E0C5F0240EC5F03400C5F0F9AAF089828A83E075F000C0AE
:20452E00E0C0F07F041201CCE0A3F5F0E0C5F0240CC5F03400C5F0F9AAF089828A83E0A382
:20454E00F5F0E0C0F0C0E07F041201CCE0A3F5F0E0C5F02411C5F03400C5F0F9AAF0898268
:20456E008A83E075F000C0E0C0F07F041201CCE0A3F5F0E0C5F0240FC5F03400C5F0F9AAB8
:20458E00F089828A83E0A3F5F0E0C0F0C0E0740675F0001260C57FF412004F74C075F08268
:2045AE00C0E0C0F0120CEC1581158174C075F082C0E0C0F074F275F071C0E0C0F07F0412DB
:2045CE0001CCE0A3F5F0E0C5F02414C5F03400C5F0F9AAF089828A83E075F000C0E0C0F0ED
:2045EE007F041201CCE0A3F5F0E0C5F02412C5F03400C5F0F9AAF089828A83E0A3F5F0E087
:20460E00C0F0C0E07F041201CCE0A3F5F0E0C5F02417C5F03400C5F0F9AAF089828A83E079
:20462E0075F000C0E0C0F07F041201CCE0A3F5F0E0C5F02415C5F03400C5F0F9AAF08982E3
:20464E008A83E0A3F5F0E0C0F0C0E0740675F0001260C57FF412004F74C075F082C0E0C042
:20466E00F0120CEC1581158102433E740675F072C0E0C0F0120CEC1581158190655AE0A3DA
:20468E00F5F0E0C5F07F041201CCF0A3C5F0F0C5F0E4F5F07F001201CCF0A3C5F0F0C5F02F
:2046AE007F001201CCE0A3F5F0E0C5F07B007C0412014D70250247DB7F001201CCE0A3F5A7
:2046CE00F0E0C5F02410C5F03400C5F07F001201CCF0A3C5F0F0C5F080C674C075F082C009
:2046EE00E0C0F0741B75F072C0E0C0F07F041201CCE0A3F5F0E0C0F0C0E0740375F000127E
:20470E0060C57FFA12004F74C075F082C0E0C0F0120CEC15811581E4F5F07F021201CCF0D2
:20472E00A3C5F0F0C5F07F021201CCE0A3F5F0E0C5F07B107C0012014D70200247C87F0288
:20474E001201CCE0A3F5F0E0C5F01201267F021201CCF0A3C5F0F0C5F080CB74C075F08283
:20476E00C0E0C0F0742275F072C0E0C0F07F041201CCE0A3F5F0E0C5F01201267F041201F0
:20478E00CCF0A3C5F0F0C5F0120134F9AAF089828A83E075F000C0E0C0F0740375F00012DD
:2047AE0060C57FFA12004F74C075F082C0E0C0F0120CEC1581158102474C740A75F000C013
:2047CE00E0C0F0120B88158115810246C67F060201E67FFE7EFF1201E812034545F07003F7
:2047EE000248201203BC7B137C0012016970030248201203BC7F011201CCF0B2977F011212
:20480E0001CCE075F0007B117C00120171600302480074C075F082C0E0C0F0742875F07261
:20482E00C0E0C0F078F5120043E60886F0C0E0C0F008E60886F0C0E0C0F0740475F00012F9
:20484E0060C57FF812004F74C075F082C0E0C0F0120CEC1581158178FB120043E60886F080
:20486E007B087C0012011418181826C5F00836C0F0C0E008E60886F054FFC5F05400C5F0D6
:20488E00D004D0032BC5F03CC5F07F001201CCF078F9120043E60886F012013418F608A617
:2048AE00F012012645F0700302492A74C075F082C0E0C0F0743475F072C0E0C0F018181822
:2048CE00860108860289828A83E075F000C0E0C0F0740375F0001260C57FFA12004F74C0E5
:2048EE0075F082C0E0C0F0120CEC1581158178F7120043E60886F012012618F608A6F0121E
:20490E000134F9AAF07F001201CCE089828A831200652B7F001201CCF002489E74C075F0FA
:20492E0082C0E0C0F0743975F072C0E0C0F07F001201CCE0F40475F000C0E0C0F0740375EC
:20494E00F0001260C57FFA12004F74C075F082C0E0C0F0120CEC158115817F020201E67FBE
:20496E00FB7EFF1201E878F9120043E60886F090959DF0A3C5F0F0C5F074E775F003C0E07A
:20498E00C0F0123FB4158115817F031201CCF0A3C5F0F0C5F090959FE0A3F5F0E0C5F045D4
:2049AE00F060137F031201CCE0A3F5F0E0C5F07B007C0012016345F07003024A9E9095A361
:2049CE00E0A3F5F0E0C5F02402C5F03400C5F07F011201CCF0A3C5F0F0C5F078F9120043F6
:2049EE00E60886F07F011201CC12006912017A7003024A9BB297742075F000C0E0C0F07F73
:204A0E00011201CCE0A3F5F0E0C5F018C396C5F00896C0F0C0E01262CF158115811581157D
:204A2E00817F001201CCF078F9120043E60886F0C0E0C0F07F001201CCE075F000C0E0C01C
:204A4E00F008E60886F0C0E0C0F01247E07FFA12004F78FB120043E60886F07F001201CCFF
:204A6E001200652BC5F03400C5F018F608A6F0181818E60886F07F001201CC1200652BC5CB
:204A8E00F03400C5F018F608A6F00249E9024AAE743F75F072C0E0C0F012127315811581B8
:204AAE00744F75F072C0E0C0F0120CEC158115817F050201E67FFE7EFF1201E8E4F5F07F1E
:204ACE00001201CCF0A3C5F0F0C5F07F001201CCE0A3F5F0E0C5F078FB12004386030886C2
:204AEE000412014D7003024B83B29712034545F07003024B8078F91200438601088602C04C
:204B0E0001C002120403D083D082F078F9120043860108860289828A83E0120087904B4489
:204B2E0002009074FFF5F07F001201CCF0A3C5F0F0C5F0024B83414B0A00314B1B00314BB9
:204B4E0003000000544B78F9120043E60886F012012618F608A6F07F001201CCE0A3F5F0D0
:204B6E00E0C5F01201267F001201CCF0A3C5F0F0C5F0024AD978F91200438601088602E428
:204B8E0089828A83F07F001201CCE0A3F5F0E0C5F07F020201E67FF57EFF1201E878FB12C9
:204BAE000043E60886F07F061201CCF0A3C5F0F0C5F018860108860289828A83E01200872F
:204BCE007B3A12007E1201717003024C2674C075F082C0E0C0F0745C75F072C0E0C0F0189D
:204BEE00E60886F0C0E0C0F0740375F0001260C57FFA12004F74C075F082C0E0C0F0120C7D
:204C0E00EC1581158174FFF5F07F001201CCF0A3C5F0F0C5F0024F0678FB120043E6088638
:204C2E00F02401C5F03400C5F07F081201CCF0A3C5F0F0C5F07F081201DAE98AF0C0E0C029
:204C4E00F0740275F000C0E0C0F012050015811581158115817F001201CCF0A3C5F0F0C561
:204C6E00F07F081201DAE98AF0C0E0C0F0740475F000C0E0C0F012050015811581158115F4
:204C8E00817F021201CCF0A3C5F0F0C5F07F081201DAE98AF0C0E0C0F0740275F000C0E096
:204CAE00C0F012050015811581158115817F041201CCF07F061201CCE0A3F5F0E0C5F01202
:204CCE0001267F061201CCF0A3C5F0F0C5F0120134F9AAF07F001201CCE0A3F5F0E0C5F019
:204CEE0089828A83F07F061201CCE0A3F5F0E0C5F01201267F061201CCF0A3C5F0F0C5F0B3
:204D0E00120134F9AAF07F021201CCE0A3F5F0E0C5F089828A83F07F061201CCE0A3F5F07A
:204D2E00E0C5F01201267F061201CCF0A3C5F0F0C5F0120134F9AAF07F021201CCE0A3F594
:204D4E00F0E0C5F07B087C0012011489828A83F07F001201CCE0A3F5F0E0C0F0C0E07F021B
:204D6E001201CCE0A3F5F0E0C5F07B087C00120114D004D0032BC5F03CC0F0C0E07F02127D
:204D8E0001CCE0A3F5F0E0C5F054FFC5F05400C5F0D004D0032BC5F03CC5F07F041201CC50
:204DAE001200652BC5F03400C5F07F051201CCF07F001201CCE0A3F5F0E0C5F07F0A12015B
:204DCE00CCF07F0A1201CCE075F0007B007C001201887012024E5F7F0A1201CCE0147F0AB4
:204DEE001201CCF080DC7F061201CC120070C001C0027F081201DAE98AF0C0E0C0F0740274
:204E0E0075F000C0E0C0F01205001581158115811581D083D082F07F061201CC1200707F66
:204E2E00051201CCE089828A831200652B7F051201CCF07F061201CCE0A3F5F0E0C5F01220
:204E4E0001267F061201CCF0A3C5F0F0C5F0024DE57F081201DAE98AF0C0E0C0F074027586
:204E6E00F000C0E0C0F012050015811581158115817F051201CC1200652BC5F03400C5F0D2
:204E8E007F051201CCF07F051201CCE07003024EEB74C075F082C0E0C0F0748B75F072C0BF
:204EAE00E0C0F07F051201CCE075F000C0E0C0F0740375F0001260C57FFA12004F74C075C6
:204ECE00F082C0E0C0F01212731581158174FFF5F07F001201CCF0A3C5F0F0C5F07F041207
:204EEE0001CCE07003024F0674FFF5F07F001201CCF0A3C5F0F0C5F07F001201CCE0A3F5B4
:204F0E00F0E0C5F07F0B0201E67FFA7EFF1201E8741175F000C0E0C0F0120B88158115818F
:204F2E00746075F065C0E0C0F0120CEC1581158174FF75F000C0E0C0F0120B881581158146
:204F4E00747B75F089C0E0C0F0746475F000C0E0C0F0124AC315811581158115817F001281
:204F6E0001CCF0A3C5F0F0C5F07F001201CCE0A3F5F0E0C5F07B007C0012014D6003025200
:204F8E00C17F001201CCE0A3F5F0E0C5F045F06014797B7A8989828A83E01200877B3A12EF
:204FAE00007E12017145F07003024FCCE4F5F07F001201CCF0A3C5F0F0C5F0024FEC741344
:204FCE0075F000C0E0C0F0120B881581158174FF75F000C0E0C0F0120B88158115817F00C5
:204FEE001201CCE0A3F5F0E0C5F045F07003024F1E747B75F089C0E0C0F0124BA4158115D7
:20500E00817F001201CCF0A3C5F0F0C5F07F001201CCE0A3F5F0E0C5F07B007C0012014D04
:20502E0060030252C1747B75F0892401C5F03400C5F0F9AAF090655AE0A3F5F0E0C5F089E2
:20504E00828A83120069C39BC5F09CC5F07F021201CCF0A3C5F0F0C5F090655AE0A3F5F0D0
:20506E00E0C0F0C0E0747B75F0892403C5F03400C0F0C0E0747B75F0892400C5F03400C506
:20508E00F0F9AAF089828A83E0120087C0E0C0F01263A17FFA12004F741175F000C0E0C064
:2050AE00F0120B8815811581746075F065C0E0C0F0120CEC1581158174FF75F000C0E0C0C5
:2050CE00F0120B8815811581747B75F089C0E0C0F0746475F000C0E0C0F0124AC31581157D
:2050EE0081158115817F001201CCF0A3C5F0F0C5F07F001201CCE0A3F5F0E0C5F07B007C58
:20510E000012014D60030252C17F001201CCE0A3F5F0E0C5F045F06014797B7A8989828A19
:20512E0083E01200877B3A12007E12017145F07003025154E4F5F07F001201CCF0A3C5F0DE
:20514E00F0C5F00252A97F001201CCE0A3F5F0E0C5F045F070030252A9741375F000C0E013
:20516E00C0F0120B881581158174FF75F000C0E0C0F0120B8815811581747B75F089C0E02A
:20518E00C0F0124BA4158115817F001201CCF0A3C5F0F0C5F07F001201CCE0A3F5F0E0C56E
:2051AE00F07B007C0012015360030252A9747B75F0892401C5F03400C5F0F9AAF07F02126E
:2051CE0001CCE0A3F5F0E0C5F089828A831200692BC5F03CC5F07F041201CCF0A3C5F0F0F9
:2051EE00C5F07F041201CCE0A3F5F0E0C5F090655A12006912017A700302526874C075F06E
:20520E0082C0E0C0F074A575F072C0E0C0F0747B75F0892401C5F03400C5F0F9AAF0898230
:20522E008A83E0A3F5F0E0C0F0C0E0740375F0001260C57FFA12004F74C075F082C0E0C053
:20524E00F012127315811581E4F5F07F001201CCF0A3C5F0F0C5F00252A97F041201CCE03A
:20526E00A3F5F0E0C0F0C0E0747B75F0892403C5F03400C0F0C0E0747B75F0892400C5F075
:20528E003400C5F0F9AAF089828A83E0120087C0E0C0F01263A17FFA12004F7F001201CC55
:2052AE00E0A3F5F0E0C5F07B007C0012016360030250A6741175F000C0E0C0F0120B881527
:2052CE00811581740A75F000C0E0C0F0120B88158115817F060201E69095ADE054107003AE
:2052EE0002530174C975F072C0E0C0F0120CEC158115819095A5E0C333F8A3E033F9908950
:20530E00DFAA82AB83E0A3FCE0A3FDE0A3FE75F003C3EC33FCED33FDEE33FED5F0F4ECF4AB
:20532E002401FCEDF43400FD0E8A828B83ECF0A3EDF0A3EEF0A3C870011914C8E94870C1F4
:20534E00229095ADE05440700302536A74EF75F072C0E0C0F0120CEC158115819095A5E03B
:20536E00C333F8A3E033F99089DF7AEE7BFF7CFFD2D5C082C083E0A3FDE0A3FEE0FFEDC371
:20538E009AFDEE9BFEEF9CFFED2400FDEE3400FEEF3400FF20D510ED251CFDEE3400FEEFC8
:2053AE003400FFD2D5801DEDC3951CFDEE9400FEEF9400FF500CED251CFDEE3400FEEF343E
:2053CE0000FFC2D575F003E4C0E0C3EF13FFEE13FEED13FDD0E013C0E0D5F0EFD0E0C4C32F
:2053EE0013F5F0D083D082E0FAEDF0A3E0FBEEF0A3E0FCEFF0A3EAC395F0FAEB9400FBEC5C
:20540E009400FCC870011914C8E9486003025380229095A5E0A3F5F0E0C5F07B007C001265
:20542E000153701078FB120043E60886F07B0C7C0012014D45F0700302546A741775F07330
:20544E00C0E0C0F0120CEC1581158174FFF5F09095A5F0A3C5F0F0C5F00256F99095ADE0A6
:20546E0054407003025488744F75F073C0E0C0F0120CEC1581158112424D9095A5E0A3FC2E
:20548E00E0FD78F91200438682088683088602088603751B8979DFE51DF0A3E51EF0A3EC99
:2054AE00F0A3EDF0A3780275F002851BA0E3C9047002051BC9F0A3D5F0F0C9047002051BF8
:2054CE00C9D8E4CC70011D14CCCAC39408CACB9400CB7800E4F0AE82AF83A3ED30E7030288
:2054EE00563E4C7003025648EB30E70302563E4A700302563EB800028003025595C01BC0F9
:20550E0001851BA0E3C9047002051BC9F8851BA0E3C92402C9C51B3400C51B7054851BA066
:20552E00E3C9047002051BC9F5F0851BA0E3C92402C9C51B3400C51B7037E8F0A3E5F0F0B7
:20554E00A3C082C0838E828F83E004F0B4FF0302557BD083D082D0E0D0E0CA24FECACB34DD
:20556E00FFCBCC70011D14CC780002563BD083D0827801D001D01BE4F0AE82AF83CA7001C3
:20558E001B14CAA302563BB801028003025635C01BC001C006C007851BA0E3C90470020573
:2055AE001BC9FE851BA0E3C92402C9C51B3400C51BFF851BA0E3C9047002051BC9F5F08578
:2055CE001BA0E3C92402C9C51B3400C51BF84F603DEEF0A3EFF0A3E5F0F0A3E8F0A3D007D2
:2055EE00D006C082C0838E828F83E004F0B4FF03025620D083D082D0E0D0E0CA24FCCACB9A
:20560E0034FFCBCC70011D14CC780102563BD007D0067800D001D01BE4F0AE82AF83CA70E7
:20562E00011B14CAA380067B007A00800D0254E99095A574FFF0A3F08016E475F004F0A342
:20564E00D5F0FBE5828583F09095A3F0A3E5F0F09095A5E0A3F5F0E0C5F07B007C0012012C
:20566E005B70030256BB9095ADE05440700302568F746575F073C0E0C0F0120CEC158115E5
:20568E008190655A12007089828A83E0A3F5F0E0C5F012012689828A83F0A3C5F0F0C5F057
:2056AE0090959FF0A3C5F0F0C5F00256F99095ADE0544070030256D6747F75F073C0E0C0C8
:2056CE00F0120CEC1581158178F9120043E60886F0C0E0C0F0E4C0E0C0E008E60886F0C0CC
:2056EE00E0C0F01261EE7FFA12004F9095ADE054407003025717749475F073C0E0C0F01266
:20570E000CEC1581158112424D9095A5E0A3F5F0E0C5F0229095ADE0541070030257407437
:20572E00AC75F073C0E0C0F0120CEC1581158112424D9095A5E0A3C333FAE033FB9089DF6D
:20574E00E0A3FCE0A3FDE0A3FEE4B297B514FBC0A8C2AFC2B3C28C8C8A8D8CC28DD28CB2A0
:20576E00B38EF0E0A3FCE0A3FDE0A3FECA70011B14CAEA4BB297308DFBC28DD5F0F670D5B1
:20578E00C2B3C28C85188A85198CC28DD28CD0A82278FB120043E60886F07B017C00120169
:2057AE004D701A18E60886F07BE87C03120169700C18E60886F07BD07C0712016345F07049
:2057CE00030257E574CA75F073C0E0C0F0121273158115810258DE78FB120043E60886F0ED
:2057EE007BE77C0312015B700302582490655EE0A3F5F0E0C5F090959DF0A3C5F0F0C5F05C
:20580E0018E60886F0C394E8C5F09403C5F018F608A6F002583890655AE0A3F5F0E0C5F034
:20582E0090959DF0A3C5F0F0C5F078FB120043E60886F0C0E0C0F0123FB415811581905816
:20584E007802009074E675F073C0E0C0F0121273158115810258DE74FD75F073C0E0C0F01A
:20586E00121273158115810258DE655800005258FFFF000084589095A5E0A3F5F0E0C5F017
:20588E007B007C0012015370030258D874C075F082C0E0C0F0741675F074C0E0C0F09095B5
:2058AE00A5E0A3F5F0E0C0F0C0E0740375F0001260C57FFA12004F74C075F082C0E0C0F045
:2058CE00120CEC158115810258DE1252E61257222274DF75F089C0E0C0F0E4C0E0C0E0742C
:2058EE00BE75F00BC0E0C0F01261EE7FFA12004F1203871203A974F4C333FA740133FB90FC
:20590E0089DFE4B297B514FBD2B2C2D5E50D60030259CEB29720B2F4C21FC0A8C2AFC28C70
:20592E00758A00758C00C28DD28C75F000201F1AB297308D07C28D05F020F30730B2F1D2DE
:20594E001F8018430A20D2D58011B297308D07C28D05F020F3ED20B2F1C21FC28CE5F0A223
:20596E008D3400F5F0AC8AAD8CC28DD28CECF0A3EDF0A3E5F0F0A320D50DCA70011B14CABA
:20598E00EB4A70A9430A40C28C85188A85198CC28DD28CD0A874F4C333FC740133FDCA7021
:2059AE00011B14CAECC39AFAED9BFBEBC313FBEA13FAE50A92E4F50A9095A5EAF0A3EBF0E0
:2059CE00742975F074C0E0C0F0120CEC15811581227FFE7EFF1201E878FB120043E608866A
:2059EE00F012014745F0700C18E60886F07BE77C0312015B45F07003025A4474C075F08270
:205A0E00C0E0C0F0743F75F074C0E0C0F074E775F003C0E0C0F0740375F0001260C57FFAAD
:205A2E0012004F74C075F082C0E0C0F0120CEC15811581025D2890655AE0A3F5F0E0C5F083
:205A4E0090959DF0A3C5F0F0C5F078FB120043E60886F0C0E0C0F0123FB4158115817B0061
:205A6E007C0012015B7003025B709095A3E0A3F5F0E0C5F090655A120069C39BC5F09CC5EB
:205A8E00F0FBACF090655CE0A3F5F0E0C5F0C39BC5F09CC5F07F001201CCF0A3C5F0F0C564
:205AAE00F09095ADE054087003025B0F74C075F082C0E0C0F0746B75F074C0E0C0F0909563
:205ACE00A1E0A3F5F0E0C0F0C0E09095A3E0A3F5F0E0C0F0C0E07F001201CCE0A3F5F0E079
:205AEE00C0F0C0E0740575F0001260C57FF612004F74C075F082C0E0C0F0120CEC1581153D
:205B0E00819095A1E0A3F5F0E0C0F0C0E09095A3E0A3F5F0E0C0F0C0E07F001201CCE0A357
:205B2E00F5F0E0C0F0C0E01263A17FFA12004F90655A12007089828A83E0A3F5F0E0C5F06C
:205B4E0012013489828A83F0A3C5F0F0C5F09095A1E0A3F5F0E0C5F09095A3F0A3C5F0F028
:205B6E00C5F09095ADE054087003025B8E74A375F074C0E0C0F0120CEC1581158112424DDF
:205B8E0074E775F003C0E0C0F0123FB4158115817B007C0012014D7003025BBD74C875F02E
:205BAE0074C0E0C0F0120CEC15811581123EF174F375F074C0E0C0F0120CEC1581158112C4
:205BCE0058DF9095A5E0A3F5F0E0C5F045F06003025BF4742B75F075C0E0C0F0120CEC15E8
:205BEE00811581025D289095ADE054087003025C12745075F075C0E0C0F0120CEC15811565
:205C0E008112424D12534F78FB120043E60886F0F51D85F01E9095ADE054087003025C41AF
:205C2E00747575F075C0E0C0F0120CEC1581158112424D9095A3E0A3F5F0E0C0F0C0E0907C
:205C4E0095A3E0A3F5F0E0C5F090655A120069C39BC5F09CC5F0FBACF090655CE0A3F5F083
:205C6E00E0C5F0C39BC5F09CC0F0C0E012541F15811581158115819095ADE0540870030222
:205C8E005CA3749B75F075C0E0C0F0120CEC1581158112424D9095A5E0A3F5F0E0C5F07BA5
:205CAE00007C001201537003025CCC74B975F075C0E0C0F0120CEC15811581025D2874C00F
:205CCE0075F082C0E0C0F074D675F075C0E0C0F09095A3E0A3F5F0E0C5F090655A1200697C
:205CEE00C39BC5F09CC5F0FBACF090655CE0A3F5F0E0C5F0C39BC5F09CC0F0C0E074037562
:205D0E00F0001260C57FFA12004F74C075F082C0E0C0F0120CEC158115817F020201E62247
:205D2E00E4F5F09095ABF0A3C5F0F0C5F0E4F5F09095A9F0A3C5F0F0C5F0E4F5F0F53285D6
:205D4E00F033748675F0019095A7F0A3C5F0F0C5F022E5328533F012014745F0600A9095FA
:205D6E00ABE0A3F5F0E0C5F045F07003025E349095A9E0A3F5F0E0C0F0C0E0122AFB1581FE
:205D8E00158145F06003025E349095ADE054047003025DE974C075F082C0E0C0F074FB751F
:205DAE00F075C0E0C0F09095A9E0A3F5F0E0C0F0C0E09095A9E0A3F5F0E0C0F0C0E07404DC
:205DCE0075F0001260C57FF812004F74C075F082C0E0C0F0120CEC158115819095A9E0A34F
:205DEE00F5F0E0C5F01201269095A9F0A3C5F0F0C5F09095ABE0A3F5F0E0C5F09095A9127A
:205E0E0000691201807003025E25E4F5F09095A9F0A3C5F0F0C5F09095A7E0A3F5F0E0C523
:205E2E00F0F53285F03322740E75F076C0E0C0F0120CEC1581158174C075F082C0E0C0F025
:205E4E00742575F076C0E0C0F09095ABE0A3F5F0E0C0F0C0E09095A9E0A3F5F0E0C0F0C082
:205E6E00E0E5328533F0C0E0C0F09095A7E0A3F5F0E0C0F0C0E0740675F0001260C57FF438
:205E8E0012004F74C075F082C0E0C0F0120CEC158115812278F9120043E60886F008E608B0
:205EAE0086F0D29778F91200438602088603088682088683E493FD740193FC2D75F0009259
:205ECE00F02CFCE5F03DFDEC2402FC74FE3DFDE4F582F583FEFFE4932EFEE43FFFC297A342
:205EEE00EA658270F1D297EB658370EAEE6CF5F0EF6DC297C5F0222278F9120043E60886A5
:205F0E00F008E60886F0D29778F91200438682088683088602088603C297E0FCC0A8C2AFA0
:205F2E00F4F000E0F4B50435E4F000E0702F7455F000E0B4552774AAF000E0B4AA1FECF04A
:205F4E0000E0B50418D297D0A8A3EAC39401FAEB9400FBEA70C2B297EB70BD8004D0A8ECE3
:205F6E00F0EA8BF02222E4F50AE475F078C0E0C0F0742E75F000C0E0C0F0125EA215811572
:205F8E0081158115819095AEF0A3C5F0F0C5F045F07003025FADE50A4480F50A025FDFE4FA
:205FAE0075F080C0E0C0F0E475F020C0E0C0F0125F0615811581158115819095B0F0A3C5E9
:205FCE00F0F0C5F045F07003025FDFE50A4480F50AA88108E4F608B880FB227FFE7EFF1210
:205FEE0001E8125F741223DB1201F3D2AF120881125D2E90838BE0600302603A745F75F041
:20600E0076C0E0C0F0120CEC15811581749675F076C0E0C0F0120CEC15811581749B75F097
:20602E0076C0E0C0F0120CEC15811581123F691212AD740175F00045F0700302609FE4A2C2
:20604E001792E0F51F7003026060B297B297B297C217122A87122C29125D60120FBF7F0054
:20606E001201CCF0A3C5F0F0C5F07B007C00120171700302609C7F001201CCE0A3F5F0E0B4
:20608E00C0F0C0E0121811158115811212AD02604074C975F076C0E0C0F0120CEC158115AB
:2060AE00817F020201E623F42581F81201B41263EC1201B402044C23F42581F886820886A6
:2060CE0083080263EC00000000000000000020202020200000000000000000000000000036
:2060EE00000000000060010101010101010101010101010101181818181818181818180132
:20610E000101010101010A0A0A0A0A0A020202020202020202020202020202020202020207
:20612E000101010101010C0C0C0C0C0C0404040404040404040404040404040404040404B3
:20614E000101010100C2D578FB120043E69060D3C2E79355F060027401A2D575F00092F06F
:20616E0065F075F0002278FB120043E6A2E7B3E4F5F092E02275F00280CB75F00480C67518
:20618E00F00680C175F01680BC75F01780B775F05780B2D2D575F05780AD75F01080A675C2
:2061AE00F00880A175F001809C75F020809778FB120043E6C0E008E6C0E012618813D0F0F0
:2061CE00D0E0500224E02278FB120043E6C0E008E6C0E012618313D0F0D0E050E924202295
:2061EE0078F7120043868208868308860708088603088604EB4C600AEFF0A31BBBFFF51CEB
:20620E0080F22278FB1200438682088683E4FBFCFFE0A3B42D030FE0A3C39430B40A005093
:20622E0012FA740A75F0001200B92AFBE5F03400FC80E4EB8CF0DF0302013E2278F91200D9
:20624E00438682088683E0600DA380FA78F91200438682088683088601088602C9C582C993
:20626E00CAC583CAE0A3C9C582C9CAC583CAF06003A380E8E5828583F02278FB12004386CF
:20628E0082088683E4F5F0FAE06009A30ABA00F805F080F4EA2278FB120043E60886F03021
:2062AE00F73A02013E78F91200438603088604088605088606ED8EF0120196401CED8EF07B
:2062CE002278F91200438603088604088605088606ED8EF012019640E4EB8CF02278FB1240
:2062EE000043860308860485FEF0E5017F0012017A600575F001E422EF0FF5F0A412017AE8
:20630E0070F6EF1475F0002278F912004386820886830886F0E0B5F0068583F0E58222A373
:20632E0070F3F5F02278F91200438682088683088601088602C9C582C9CAC583CAE0F5F06D
:20634E00A3C9C582C9CAC583CAE0B5F0056009A380E37401500274FF0200871263C312636E
:20636E00CF1263D61263DDE0F7A30980F71263C31263D61263CF1263DDE7F009A380F71284
:20638E0063C31263CF1263D6A8821263DDE6F7080980F71263C31263CF1263D61263DDE060
:2063AE00A3CAC583CAC9C582C9F0A3CAC583CAC9C582C980E778FA120043860418860318BE
:2063CE00228683188682182286021886011822EB4C60061BBBFF011C221581158122126553
:2063EE0033868208868308E4FEFFE07006126533E4F022B42551A3E0B42D05430780A3E084
:20640E00B4300343074024D0B40A00500BCE75F00AA42EFEA3E080EEE0B46413E60886F083
:20642E0030F70843072012013EA6F018F68003B4750543070A8021B478054307108019B442
:20644E006F104307088011126533F0A3126533A38095B462624307027A00C004C005C006A0
:20646E00C007AB0753031F7C00E60886F01200D3A6F018F6EDD007D006D005D0042430B46C
:20648E003A0040022407C0E00AE645F070CC126533A902EF30E505742DF0A30A12653CD027
:2064AE00E0F0A3D9FA0808EF30E7A1EAC39E509C7420F0A30A80F4B4630DAA01126533126A
:2064CE00653CE6F0A380DEB47331C082C08386820886837A00E06004A30A80F986831886B5
:2064EE008212653312653C126533E0A31265336004F0A380F2D005D00480AAB4691B8601DD
:20650E007A00E76004090A80F912653312653C8601E76091F009A380F8F97A01126533121C
:20652E00653CE9809ECDC583CDCCC582CC22EE601A8FF020F715C002EAC39E500C74203082
:20654E00F6027430F0A30A80EFD0022200A0F05F0078484558203E004952302000EE654366
:20656E006F6E736F6C652073746174757320666C61677320253032780A00205472616E733B
:20658E003A20204865616420253032782C205461696C20253032782C2043747220253032D1
:2065AE00782C204D617820253032780A00205265633A202020204865616420253032782C09
:2065CE00205461696C20253032782C2043747220253032782C204D617820253032780A00B5
:2065EE0030313233343536373839414243444546003030200020002A2A2A20426164206323
:20660E006865636B73756D3A202532780A002A000A002A2120004F4B0A003E002A2A2A202A
:20662E004E6F206164647265737320737472696E672E2E2E0A004E65742061646472657384
:20664E00732069732025730A004E65742061646472657373205B25735D002E2020537461C8
:20666E00636B207573656420253032782F253032782E0A004572726F7220666C6167732091
:20668E00253032782E20204E6574776F726B20636865636B73756D206572726F7273202520
:2066AE00750A004C6F6767696E67206D6F64652069732025750A004E6574206D6F646520F5
:2066CE0069732025750A002A2A2A204E20636D642073796E746178206572726F720A002A87
:2066EE002A2A20556E6B6E6F776E20636F6D6D616E643A205B25735D0A0042616467652082
:20670E00726573706F6E73652064656C6179206973202575207469636B730A002A2A2A2031
:20672E004261642043616C69627261746520636F6D6D616E640A002A2A2A20556E6B6E6FEB
:20674E00776E2048455820636F6D6D616E640A002A2A2A20426164676520706F6C6C696E19
:20676E006720696E74657276616C20666F7263656420746F2025750A004261646765207062
:20678E006F6C6C696E6720696E74657276616C206973202575207469636B730A002A2A2A65
:2067AE00204F75747075743A2020626164206269742049440A002A2A2A204F757470757434
:2067CE003A202062616420666F726D61740A004E756D626572206F66206261646765732053
:2067EE0069732025750A002A2A2A2051756572793A202062616420706172616D0A004553C3
:20680E004554002A2A2A20556E6B6E6F776E20636F6D6D616E640A002A2A2A204D69737300
:20682E00696E6720706172616D657465720A0044757479206379636C6520636F72726563AD
:20684E0074696F6E206973202575206379636C65730A002A2A2A204D697373696E67204D28
:20686E00434952207265636F7264206E756D6265720A00417661696C61626C6520636F6DFA
:20688E006D616E6473202876616C75657320696E20646563696D616C20756E6C657373203F
:2068AE006E6F746564290A00202874696D657320696E20352E3136206D73207469636B73F4
:2068CE00290A0020413D737472202020202B20736574206E6574776F726B2061646472651F
:2068EE0073730A002042206E202020202020202073657420626164676520726573706F6E94
:20690E0073652074696D652064656C61790A00204352206E2020202020202073686F772085
:20692E004D43313435303330206F736320706572696F642C206E203D207265706F72742091
:20694E0064657461696C0A0020435420202020202020202063616C69627261746520747228
:20696E00616E736D6974206F7363696C6C61746F72202855312E313120746F205431290AE8
:20698E0000204420202020202020202A2064756D7020696E7465726E616C207374617475B7
:2069AE0073207661726961626C65732028736F6D6520696E20686578290A0020452020202D
:2069CE0020202020202A2073686F7720616E6420636C656172206572726F7220666C616780
:2069EE00730A002049206E202020202020202073657420626164676520706F6C6C696E67A1
:206A0E0020696E74657276616C0A0020484420616464722020202064756D70204D434952F1
:206A2E0020646174612066726F6D2052414D20746F2048455820772F626173652061646408
:206A4E00720A0020484520202020202020202061732048442C206275742066726F6D20458F
:206A6E0050524F4D0A0020485220202020202020202072656365697665204D434952206434
:206A8E006174612066726F6D2048455820746F2052414D0A00204C206E20202020202020F2
:206AAE0020736574207265706F7274696E67206D6F646520286269746D6170706564290A6C
:206ACE0000204E206E20202020202A2B20736574206E6574776F726B206D6F64650A002032
:206AEE0050206E2020202020202020736574206E756D626572206F6620626164676573201A
:206B0E00746F20706F6C6C0A0020512020202020202020202064756D7020616C6C207265EC
:206B2E00636569766564204D4331343530333020494420636F64657320696E206865780AB9
:206B4E00002051206E202020202020202064756D702073696E676C65204D43313435303323
:206B6E003020494420696E2062696E6172790A002051206E2D6E20202020202064756D7074
:206B8E002072616E6765206F66204D433134353033302049447320696E206865780A002042
:206BAE005245534554202020202020706572666F726D20706F7765722D6F6E207265736563
:206BCE007420696E697469616C697A6174696F6E0A002053206E2020202020202020736548
:206BEE006E64204D4331343530333020495220494420636F6465206E0A0020534D206E20AF
:206C0E0020202020202073656E64204D434952207369676E616C206E2028312D3939392014
:206C2E0052414D2C20313030302D31393939204550524F4D290A002054206E2020202020D8
:206C4E00202020747261696E206E6577204D43495220636F64652C2073746F726520696EC8
:206C6E002052414D206173206E2028312D393939290A00205444206E202020202020207367
:206C8E0065742064757479206379636C6520636F7272656374696F6E20666163746F7220E0
:206CAE00302D3235350A00205458202020202020202020636C656172204D434952206461A0
:206CCE0074612066726F6D2052414D0A002B206D61726B73206E6574776F726B2D6F6E6CEA
:206CEE007920636F6D6D616E64730A002A206D61726B7320646562756767696E6720636F6B
:206D0E006D6D616E64730A0054726E202575205B25303478206865785D0A00526376202535
:206D2E0075205B25303478206865785D0A0020253033753D25750A0020253033752D2530EB
:206D4E0033753D002530327800495220696E74657266616365207374617475733A0A0020AD
:206D6E004952537461746520253032782C20495265635374617420253032782C204261648D
:206D8E006765446C792025752C2042616467655273702025750A00204952437472202530C5
:206DAE0032782C2000494E756D53656E6420253032782C20495242697473302025303278E5
:206DCE002C2054305469636B7320253032780A00205472616E733A20204865616420253025
:206DEE0032782C205461696C20253032782C2043747220253032782C204D61782025303239
:206E0E00782C20005B494F7574486561645D2D3E253034782C20005B494F75745461696CD7
:206E2E005D2D3E253034780A00205265633A202020204865616420253032782C2054616982
:206E4E006C20253032782C2043747220253032782C204D617820253032782C20005B49493B
:206E6E006E486561645D2D3E20253034782C20005B49496E5461696C5D2D3E202530347821
:206E8E00002D2D2D20436F6E6E656374205531312E3120746F20543120696E7075740A003B
:206EAE00202020202043656E74657220257520487A2C2072616E676520257520487A2C20E6
:206ECE00737465702020257520487A0A0020202020507265737320616E79206B6579207430
:206EEE006F20717569742E2E2E0A0025367520487A205B003C3C3C20756E646572202575C5
:206F0E005D0A006F766572202575203E3E3E5D0A005D0A002D2D2D20446973636F6E6E6504
:206F2E006374205531312E312066726F6D20543120696E7075740A002D2D2D205472696726
:206F4E006765722072656D6F746520756E697420666F722065616368206D6561737572652F
:206F6E006D656E740A0020202020204D4331343530333020636C6F636B2069732031362F0A
:206F8E0028626974206672616D652074696D65290A0020202020507265737320616E79203A
:206FAE006B657920746F20717569742E2E2E0A002053616D706C6520253275207261773DEB
:206FCE00253034783D25357520006376743D253034783D2535752075730A00204573742061
:206FEE00626974206672616D652061646A75737465642066726F6D20257520746F2025755A
:20700E002075730A0020426974206672616D652074696D65207468726573686F6C64733A7D
:20702E0020002575200075730A002053616D706C652025327520253575207573002C20675E
:20704E006C697463682069676E6F7265640A002C20756E757365640A002C206C6F6E6720F6
:20706E0073706163652069676E6F7265640A002C2025752068616C662D6672616D65732078
:20708E002D3E2025752075732F6672616D65200020426974206672616D652074696D652002
:2070AE0069732025752075730A004E6F206461746120696E2052414D2C20696E69746961E2
:2070CE006C697A696E6720656D707479207374727563747572650A00495220646174612036
:2070EE00617420253034782C207365656B696E67207265636F72642025750A002D2D2D2050
:20710E0044756D70206265666F7265206465636F6D7072657373696F6E0A002D2D2D2044A8
:20712E00756D70206166746572206465636F6D7072657373696F6E0A004D434952207374E6
:20714E00617475733A0A0020704D43446174613D2530347820704D43546869733D253034CA
:20716E007820704D434E6578743D25303478200A00204D43526563733D25303478204D4337
:20718E0052656349443D25303478204D4350756C7365733D253034780A0054696D65722067
:2071AE006275666665720A0020253032782530347820253032782530347820002025303236
:2071CE00782530347820253032782530347820002025303278253034782025303278253054
:2071EE00347820002025303278253034782025303278253034780A0052414D207265636FC2
:20720E0072642073746F726167653A0A00202530347820002025303278003A253032782573
:20722E003034783030002530327800253032780A002A2A2A204E6F20495220646174610A22
:20724E00003A303030303030303146460A002A2A2A20496E74656C20484558206C696E6568
:20726E00206D757374207374617274207769746820636F6C6F6E0A5B25735D0A002A2A2AD0
:20728E0020436865636B73756D206572726F723A20253032780A002A2A2A204C696E65209A
:2072AE00616464726573732062656C6F772073746172743A20253034780A00436F6E7665F3
:2072CE007274696E6720746F2074696D65722072656C6F61642076616C7565732E2E2E2047
:2072EE00002020436F6E76657274696E672066726F6D2074696D65722063617074757265F8
:20730E002076616C7565730A002A2A2A204E6F2070756C73657320746F20636F6D707265E5
:20732E007373206F722052414D206973206F6276696F75736C7920746F6F2066756C6C0A01
:20734E00005374617274696E6720636F6D7072657373696F6E0A00496E6372656D656E7452
:20736E00207265636F726420636F756E7465720A0052656D6F76696E6720626164207265B1
:20738E00636F72640A002020636F6D7072657373696F6E2066696E69736865640A002D2D6D
:2073AE002D2044756D70206265666F7265207472616E736D697373696F6E0A002A2A2A2057
:2073CE00426164204D434952207265636F7264206E756D6265720A002A2A2A20495220643E
:2073EE00617461206E6F742076616C69640A002A2A2A204952207265636F7264206E6F7455
:20740E0020666F756E640A002A2A2A204E6F2070756C7365733A2025640A002020526177AA
:20742E002064617461206361707475726564210A002A2A2A205265636F7264206E756D6212
:20744E006572206D757374206265206265747765656E203120616E642025750A0052656DE1
:20746E006F76696E67207265636F72643A20704D4354686973202530347820704D434E6556
:20748E0078742025303478204C656E67746820253034780A002D2D2D2052414D2062756640
:2074AE0066657220726561647920666F72206E6577207369676E616C0A002A2A2A2053746E
:2074CE006F72696E67206669727374207265636F726420696E206E65772073747275637472
:2074EE007572650A002D2D2D2053656E64207369676E616C2066726F6D2049522072656D66
:20750E006F74652C20707265737320456E74657220746F20717569742E2E2E0A004E6F2027
:20752E0070756C7365732073746F7265642C20636170747572652063616E63656C6C6564F5
:20754E000A002D2D2D2054696D657220627566666572203D2063756D756C617469766520F5
:20756E0074696D65730A002D2D2D2054696D657220627566666572203D20696E6372656D94
:20758E00656E74616C2074696D65730A002D2D2D204E6577207369676E616C2073746F7226
:2075AE00656420696E2052414D0A002A2A2A20436174757265642064617461206E6F742042
:2075CE0073746F7265640A00546865726520617265202575206279746573206F6620524109
:2075EE004D20617661696C61626C650A00506F6C202575205B25303478206865785D0A0038
:20760E00426164676520706F6C6C696E67207374617475733A0A0020506F6C4E756D494464
:20762E00732025752C20506F6C4E65787449442025752C20506F6C6C446C792025752C20A0
:20764E00506F6C6C496E74657276616C2025750A000A4D4349522D4C696E6B204E657477CE
:20766E006F726B6564204952204170706C69616E636520436F6E74726F6C6C65722C205699
:20768E00657273696F6E2000312E3166000A2020436F7079726967687420313939322C20F2
:2076AE003139393420436972637569742043656C6C61722C20496E632E0A002D2D2D2046F4
:1576CE00656C6C206F75742074686520626F74746F6D210A00B1
:00000001FF
